:020000041100E9
:10300000002373B52B4D2C4C28006361022601F080
:1030100069FA4021FE2221742800284B009601F015
:10302000B3FA002836D1217CFF222800244B0096D9
:1030300001F0AAFA00282DD1224BA2899A4226D16A
:10304000E389214A93420DD1204B6361204B2268D2
:10305000002A03D1002B01D043CB43C4280001F048
:103060007FFA73BD1B4A934201D00023EFE71A4B4E
:103070001A4A1B68934206D9C02304222800217CE7
:103080009B0001F0F7FA114B6361154BDFE700235A
:103090002374EAE7CC233821AC2228009B01217459
:1030A00001F0E8FA0028F2D10E4B63610E4BE38188
:1030B0000E4BCCE7BC44FF1F7064FF1F7C64FF1FF6
:1030C0007E64FF1F59590000830500001143001161
:1030D00094BF0011821500009464FF1F8713000045
:1030E000A0BF0011C9430011AAAAFFFF88BF0011A9
:1030F000F7B5164B0192C318021D002000938823D8
:103100005B05D3181B685C1C1AD09CB2402C18D8E5
:103110008D781E0CAC466746CD782D023D43AE42FD
:1031200006D1019800280ED110000C70240A4C70B2
:1031300003249BB20733A343D218009B9A42DED3E9
:10314000FEBD4432F9E71000FAE7C046FC0F00006C
:10315000802213B503000324019189B25201073183
:103160009B18A14304305A1A88235B05C3181B68B7
:10317000591C03D190429241104016BD99B240298A
:1031800007D80B000733A343C0189042ECD30020AC
:10319000F3E74430F9E7134B134A1B68126810B584
:1031A000FA24934201D81A00F824104BE4021B6859
:1031B0009A4210D813000E4A12689A420ED3013375
:1031C00007D1F823DB029C4203D10A49054808F0E5
:1031D00087FB200010BDFC24E402ECE7FE24E4029F
:1031E000F7E7C04600C0071100D0071100E0071143
:1031F00000F00711FFFFFF7FF0B59BB015000490B2
:103200000391402A00D9A0E006AB59801A80FFF74D
:10321000C2FF0400042816D9002206A9FFF768FFA0
:10322000052810D906AB1B88AB420CD1002D07D066
:10323000514B2A000499C01808F0FAFA002802D16C
:1032400001201BB0F0BD06AB1D8020000699FFF7E2
:103250007FFF041E7BD1069B0793FFF79CFF802313
:103260005B01C618802307001B039E4201D3F8268A
:10327000F60288235B05F31801931B68013302D023
:10328000019808F04DFD3D49019808F029FB3B1DD0
:103290000293331D05938822029B52059B181B68DD
:1032A00008935A1C3CD044219AB20091402A04D879
:1032B0000320D11D814389B2009103991B0C8B42DD
:1032C00024D0402A22D80122300008A9FFF710FF9D
:1032D000021E1BD1380008A9FFF70AFF04000428CA
:1032E00031D9009A059B9B1880225201B218934253
:1032F00040D288235B05C118009A09A808F048FC51
:103300001D4B009A09A9F01808F012FD009A029BC3
:103310009446634402931A4B029AFB189A42BAD31A
:1033200088235B05FC1821680198013908F0D8FA58
:10333000200008F0F5FC039A07AB5A80300007998B
:10334000FFF706FF0400002C03D1002079E70428D2
:10335000FBD988235B05E018069908F0C1FA03231E
:10336000EA1C9A4300D16BE7034B0499E01808F07C
:10337000DFFC65E70424ECE704000011FFFFFF7F9A
:10338000F80F0000F7B505001400402A21D80027E7
:1033900001AE71803780FFF7FEFE042816D93A008F
:1033A0003100FFF7A5FE042810D93688BC420BD0A7
:1033B000BD4209D0221CB44200D9321C064B92B245
:1033C000C118280008F0E4FB30B2FEBDC04300B2D3
:1033D000FBE703204042F8E70400001137B5042260
:1033E00004000D0001A81649FFF7CCFF02000428D5
:1033F0000BD1019BA34208D3AB4204D0104901A8D2
:103400000195FFF7F9FE01203EBD0E4C2368200018
:10341000019308F085FC019920000139019108F021
:103420005FFA80235B01E418074B9C42EED1042233
:10343000034901A80195FFF7DFFE0020E4E7C0463D
:103440005555000000C007110000081130B589B0C3
:1034500008F0E6FB10226946254808F001FD254BDF
:10346000009A9A420ED1019B029A0F2B33D8002169
:1034700001240698013B08D2002900D00292029B49
:10348000013331D10023029325E0551CF2D1020013
:103490002100EFE710341022200004A908F0E0FC1E
:1034A000029B013301D1069B0293882304995B059B
:1034B000C918059B06981A03120B049105928142C4
:1034C00003D02B4201D108F063FB019B013B019328
:1034D000019B002BDED1029B002B03D004930498A8
:1034E0004168084709B030BDE025014C2D03EFE7E6
:1034F0000000011150485936F7B50F4F0F4BFA6DC8
:1035000004001A4084235B001343FB65030010335F
:10351000019300252E00112008F0B2FA0322BB6EA1
:103520001340AB4002351E43202DF4D1019B40C413
:10353000A342EED1F7BDC04600F0004000FEFEFF02
:10354000802270B5AD4CAE4BD200002120001C6033
:1035500008F0DEFA2300AB4A88331A60AA4B1A78C7
:103560006E23002A00D01133E3620A232365A74BA0
:103570001878A74BA0630138E361C3B2032B01D8CD
:1035800010232362A34B37226361C823DB00A361AE
:1035900023008C331A60082336210F3AE518E163C3
:1035A00023646264E9670439251DE96725003B2629
:1035B000BC352E602500C0352B602500C4352A603F
:1035C00025000636CC352E602500083EC8352E6015
:1035D0002500D03529602100D4310B602100D8317D
:1035E0000A6021000225E0310D6025004221DC3512
:1035F000296025001B3EE4352E602500E8352B6050
:103600002500EC352A6022000525F43215602200E1
:10361000F032116022001831903211602200943291
:10362000136023003C2298331A60AF23DB00236031
:10363000794B2363032805D808F03AF9330235376C
:103640001523636096232100FA225B00A360E360E8
:10365000C8332361714BFC319200A3640A6062623B
:103660006F4A704DA2627322E2656D3A6265A2658F
:103670000232E5644A600221616696218900A166F2
:10368000626709210022E166A2676749674A684EBE
:103690002167E2673560032811D808F009F9960818
:1036A0009EA61023CDE70E23CBE70C23C9E720000D
:1036B0001A259C30056020000735A03005602000E9
:1036C000A83003602300FA20F8338000186023003C
:1036D0006420A433186023005F38AC3318602300E3
:1036E0000338B03318602300C630B43318602300A9
:1036F0000020B833186023003825FC339D604D4D01
:103700005A665D644C4D9A64DD619625AD001D627C
:103710004A4D9A675D62F53DFF3D9D621E25484A10
:10372000DD6618675867D9651966DA67BE23C02158
:10373000444A5B00E250444B4900635004316250FC
:10374000C4225200A350FA23E4205B000432A350A9
:103750000432A3503D493E4A3E4BD1603E49800071
:1037600019503E49E938FF3819503D490430195085
:103770003C491038D1613C4911633C4951633C4993
:1037800011603C49195019003B48F83108603B4929
:10379000D16582213A4A89005A501A0039490832C3
:1037A000D1671A003849B43211608821374A89003C
:1037B0005A501A00364988321160364ADA6408F0E5
:1037C00057F9012008F054FA70BD200014259C30F0
:1037D000056020000435A03070E7200010259C30E3
:1037E000056020000335A03068E720000E259C30DE
:1037F000056020000235A03060E7C0460004FF1FCE
:103800004867FF1F4072FF1F0447FF1F4A0AFF1F40
:103810003A07000080C3C9019A02000050C30000AB
:103820006A180000280A0000204E000088130000DB
:10383000F009FF1F001F001168100000C4090000FC
:10384000DC05000040420F0010270000FD1BFF1F99
:10385000FC00FF1F0000FF1F012FFF1F2932FF1F69
:10386000C130FF1FD51FFF1FF11FFF1F9D21FF1F2D
:10387000491FFF1FC128FF1F692CFF1FD918FF1FF9
:10388000CD27FF1F3525FF1F4125FF1F491EFF1FA5
:10389000011FFF1FC11DFF1FF7B50B0CFF270122E2
:1038A000009300233C001E001D009446019089B245
:1038B00062469A401000084018413618B6B2FF2FF1
:1038C00002D1012E00D19FB2009802401A41AD18DA
:1038D000ADB2FF2C02D1012D00D19CB20133102BCF
:1038E000E6D10320012E07D1012D04D1019B240133
:1038F000E4191C700138FEBD102EFCD10238102DC9
:10390000F9D00230F7E710B5064C2378002B07D129
:103910000548FFF7F1FD0548FFF7EEFD0123237091
:1039200010BDC0460A67FF1F1C67FF1F0C67FF1F03
:10393000F0B58BB00D0001230190102936D8FFF7A8
:10394000E2FF00231A001B48C15C01335218102B00
:10395000FAD1023B002A29D0174B184C1F680023CC
:1039600006A9E25C1600FA5C56405E540133102B47
:10397000F7D102AA08F02CF82A0002A9019808F051
:103980004FFA08F005F823681B18236008F000F8C8
:1039900063681B18636007F0FBFFA3681B18A36034
:1039A00007F0F6FFE3681B18E360002318000BB074
:1039B000F0BDC0461C67FF1FA445FF1F0C67FF1F1B
:1039C000F0B502250124614B91B01D700293604B4C
:1039D000604E1C70604F0393336800212800BB7059
:1039E00006F008FE280006F0FFFC0023984205D0F0
:1039F000BA78552A02D0332A00D09AE033600020EA
:103A000006F060FF08F05CF8FFF79AFD07F018FF7A
:103A10001F2201240021514B36251A70504B1C7077
:103A2000504B1970504B19689143163A0A431A606B
:103A3000602219689143403A0A431A6008F0B8F9C5
:103A400007F05EFFC120FF21484B80001A588A43CF
:103A50001A50C522920098588843BF3901439950A3
:103A60009858434908408021C9010143802099505A
:103A70009958C0050902090A0143995080213D481F
:103A8000490108F06DF80323220000933A4901949C
:103A90003A4807F0BDFE2E22394904A808F078F80C
:103AA00002AB04ACED1861782078023406F0BCFC5F
:103AB000A542F8D1334C344B226803201A40A0238E
:103AC000DB0213432360802322689B04134323609B
:103AD00022682E4B1A4080239B03134323602C4AF9
:103AE0002C4B934200D8012008F042F807F020FF49
:103AF00080232268DB0413432360029B187808F0BC
:103B00001FF9039B1878C0B207F08AFF07F0C8FFBF
:103B10002149042007F04CFF06F0A0FE00F0B6F8A3
:103B200000F0FEFD00F090FE00F01EFA002011B043
:103B3000F0BD00932100184A042008F089F8802382
:103B4000DB059C62FFF782FC59E7C0464A0AFF1F6B
:103B50000447FF1F34F00040A064FF1F480AFF1F06
:103B6000490AFF1F680AFF1FBCF0004000E100E0A7
:103B7000FF00FFFF0847FF1F8C59FF1F0857FF1F5B
:103B8000B0BE001114F00040FF7FF8FFFFFF9FFF61
:103B90000080FF1F4072FF1F3B00010870B5002529
:103BA00029492A4A2A484D6308CA1B051B0DED18EE
:103BB0008242F9D10022274B8B63274B08211A62DE
:103BC0008022264B9205DA67254BDA688A43DA6051
:103BD000244A1278012A03D09A6823490A409A603D
:103BE00000260121214C11202660DA688A43DA6020
:103BF00008F006F8112008F053F9636C1C4A1340D2
:103C000063641C4C1C4A6C43200C040064239042E7
:103C10000AD8FA223300D200904205D9174B0A2164
:103C2000C01808F025F9C3B2154A11201372D480C8
:103C300007F06EFE134B1B78002B04D1124B1021A2
:103C4000187807F03DFE70BD00000540880705406C
:103C500000080540FF01000000F0004004E100E022
:103C60003CF000404A0AFF1FFFDFFFFF0038004022
:103C7000FFFDFFFFAE060000B70B000030F8FFFFAE
:103C80008864FF1FC266FF1FC064FF1F002210B5BB
:103C90001100112007F0ACFE10BD0000F8B50023A4
:103CA000012508263A4F3B4C3B62E3681120AB43A9
:103CB000E360E368B343E36008F0F2F8112007F033
:103CC0009FFF112007F03CFF40232268022113438D
:103CD000236080236268DB02134380226360A36851
:103CE00009201343A360A3682B4A1340A3608023D9
:103CF000A2689B0113431022A360236C93432364A7
:103D0000236C2B43236480235B013B62226B234B98
:103D10001A402263626B1A406263A26B1A40A2636C
:103D2000E26B1340E3631E4AE3681340E36006F06E
:103D30007BFB2900092006F08BFC8023194A9B009D
:103D4000516C11200B43536407F012FEFD21164BFA
:103D5000164A89005A508023C720E26B5B03134345
:103D6000E363E36880001E43E660E368104A1D4396
:103D7000104BE56019581140802212020A431A5074
:103D8000802292051A6080220B4B5A63F8BDC04610
:103D900000F000403CF00040FFFFDFFFEFFFEFFFCF
:103DA000FFFF7FFF003800400000FF1F9D3B001118
:103DB000FF00FFFF00E100E00000054030B503A870
:103DC00004880B20002C0ED14968074D08784978EB
:103DD000090201430A20A94205D1012120001980CE
:103DE000024B1B7A137030BD192A00008864FF1F34
:103DF000F7B5150008AA16884A680F4F147852784C
:103E0000120222430A24BA4214D10122DBB20192E7
:103E100000962A0007F072FC041E0BD1074B1B68AA
:103E2000002B07D068782A780002104342425041A4
:103E3000013098472000FEBD022900000C64FF1FDE
:103E400030B5012503790400BFB02B4212D00A49D6
:103E5000408806F0BFFF28420CD06A46074B6946EF
:103E60005B8D55801380064B60881B7A137100228E
:103E700004F0A2F83FB030BD0464FF1F3043FF1FC1
:103E80008864FF1F10B50549054806F059FF042155
:103E9000044A054806F016FF10BDC0460464FF1F23
:103EA000FFFF0000E0BE00113043FF1F10B50248C5
:103EB00004F004FF10BDC046413E0011062310B5BA
:103EC000837010330371443B43712A33837144334D
:103ED000C37100230222012103720E4B0270417054
:103EE0001C8881724472197A0273C1729A78427383
:103EF000DA7882730322C2731A7902745A7942748F
:103F00000C2282749A79C274DB7903751123C37011
:103F1000152010BD8864FF1F10B5122007F0E8FDC2
:103F2000104B12220021186007F0F2FD002007F06C
:103F3000CFFE012007F084FF022004F063F9032084
:103F400006F078F9042003F0A1FB052004F06EF8D8
:103F5000062001F033FA072006F094FE082001F055
:103F60001BF810BD1064FF1F10B507F009FD0120FC
:103F700007F036FE07F06CFD002010BD094B10B5B0
:103F80000400984205D0012904D12000064906F01A
:103F9000D7FE10BD0229FCD1013904F04DFE0028E6
:103FA000F3D0F6E7FEFF00003664FF1F70B50D7A10
:103FB000100004AA2C00168810221440154220D1AB
:103FC000002E20D10A78022A18D14A685178157833
:103FD0000E4A09022943914205D00D4A914209D067
:103FE0001C800A2404E014220A491A8007F0D0FD3C
:103FF000200070BD0C2208491A80F7E71C800124BC
:10400000F6E70824F4E70B24F2E7C046F3FF0000CC
:10401000F4FF00008845FF1FB8BF001110B5040071
:104020000749084806F08CFE074804F087FD002089
:10403000E40704D50721054A054806F043FE10BDF4
:104040003664FF1FFFFF00007D3F001120BF0011FD
:104050007443FF1F00B50C4BBFB01A780B4901A881
:1040600000F0ACFC6B4680B25880002809D06A464C
:10407000074B69461B881380064B0022188803F003
:104080009BFF3FB000BDC0461464FF1F1564FF1FB7
:10409000CE43FF1FD844FF1F00B50C4BBFB01A78AA
:1040A0000B4901A801F0CEFE6B4680B25880002873
:1040B00009D06A46074B69465B8D1380064B002288
:1040C000188803F079FF3FB000BDC0463E64FF1F73
:1040D0003F64FF1F7443FF1FD844FF1FF7B50E0056
:1040E000377A1C0008AB11003D001A8820231D40C0
:1040F0001F423CD13378022B3BD173681F785B7829
:104100001B023B431E4FBB4208D01E4FBB4214D084
:104110001D4DAB4221D00A252800FEBD002A2AD120
:10412000142C2AD82200F06807F032FD174B1C70BF
:10413000012CF1D9FFF7B0FFEEE7002A1BD1202CAC
:104140001BD82200F06807F023FD114B04211C70DE
:10415000104B187807F0B4FBDEE7E3B201240092BD
:1041600001940A00310007F0C9FA0500D4E70825D8
:10417000D2E70125D0E70B25CEE70D25CCE7C046D9
:10418000F3FF0000F4FF0000022900003E64FF1F5F
:104190001464FF1FC064FF1F332310B504000370B5
:1041A0000A220749013007F0F3FC064B0F201B6879
:1041B0001A0AE37222731A0C1B0E6273A37310BDEA
:1041C0008864FF1FB064FF1F30B501250379040028
:1041D000BFB02B4213D00B49408806F0FBFD2842AC
:1041E0000DD06A46084B01A81B881380FFF7D4FF47
:1041F0006B46588000226946608803F0DDFE3FB0C0
:1042000030BDC0463664FF1FCE43FF1F10B50248C5
:1042100004F054FD10BDC046C941001170B5160030
:1042200004AA148805AA15784A6850781178000203
:104230002A4A0843801805284BD807F039FB031396
:104240001E29343F0720032C0BD80422121BAA423C
:1042500000D92A0022491A803000091907F098FC79
:10426000002070BD0720112CFBD81222121BAA427D
:1042700000D92A001B491A80EEE707200E2CF0D83F
:104280000F22121BAA4200D92A0017491A80E3E71D
:104290000720032CE5D80422121BAA4200D92A00C9
:1042A00012491A80D8E70720032CDAD80422121BFF
:1042B000AA4200D92A000E491A80CDE70720032C14
:1042C000CFD80422121BAA4200D92A0009491A8019
:1042D000C2E700220A201A80C3E7C046DCD5FFFFF0
:1042E0006BBF00115C64FF1F5BBF001156BF001164
:1042F00051BF00114CBF001110B50D21024A0348F7
:1043000006F0E0FC10BDC04640BF0011E443FF1FB3
:10431000F0B50024274E85B03000B47100F0E2F80B
:10432000254D264BEA89297C9A422FD1042330005F
:1043300003AA00F057F90400300000F011F901233E
:10434000B371002C34D16B4699892B68C9BA4B43A1
:1043500029891B4A1B145B1853806B46D9896B68EB
:1043600049BA89B24B4369891B0C5B181548191C63
:104370001BB2834200DD011C0B0400D50021138811
:10438000918001331380200005B0F0BD0227220088
:1043900003AB3000009700F0F7F80E230400297CEF
:1043A0000122300000976B4400F0EEF80443C3E7AD
:1043B0001C00E8E7BC44FF1F7064FF1F830500007A
:1043C0008864FF1F0F27000073B5234E300000F0F4
:1043D00089F8224D07236A463000297C00F002F953
:1043E00004003000002C33D16B461B787F2B2FD874
:1043F00000F0B6F86B46D878F02302041B031A408D
:104400006B469B8816495BBA9BB21A432B6800091E
:1044100053432A891B0C9B184B806B465A789B7818
:1044200012031B011A436B68024353436A891B0C36
:104430009B180C481A1C1BB2834200DD021C13049B
:1044400000D500220B888A8001330B80200076BDC6
:1044500000F086F80124F9E7BC44FF1F7064FF1FD9
:104460008864FF1F0F27000070B5114C237C002BC0
:104470000FD0382B0ED10F4D280000F033F8CC238D
:10448000AC222800217C9B0100F0F4F8280000F009
:1044900067F870BD084BE2899A42FAD1054D2800B1
:1044A00000F020F800222800217C00F0C5F8EDE79C
:1044B0007064FF1FBC44FF1F8305000010B5084B4C
:1044C0001A7C002A09D05B69002B06D09847041E8D
:1044D00001D0FEF795FD200010BD0124F9E7C0468C
:1044E0007064FF1F70B5C17905000C00631E9C410C
:1044F0001A4BE402E41849000460C9B2007906F0DE
:10450000DDF8E979687949000131C9B206F0D6F8D9
:10451000E8790930C0B207F013FB0023E36661338A
:104520002360AA795B3B002A0ED022689A43023BA3
:10453000134323600A23E3610733236200232363C9
:10454000A3630133E36370BD22689A4302231343DC
:104550002360462363610633A361EFE70050004008
:1045600070B5002504000368DD66C0790930C0B26B
:1045700007F096FC2900207906F03CF829006079C4
:1045800006F038F870BD0000F8B51E0006AB1D78C7
:10459000002304681700E366616007F041FB012314
:1045A0008022E3662B0027615200013B08D207F00E
:1045B00077FB08200A4A1168002D03D12800F8BDB6
:1045C0002261F2E7236F034203D02369013D337078
:1045D000013613685B1A032BEED90125EEE7C046BE
:1045E0006008FF1F70B51C00002305681600EB660D
:1045F000696007F015FB01238022EB66230052005F
:10460000013B08D207F04CFB08200A4A1168002C35
:1046100003D1200070BD2A61F2E72B6F034203D063
:104620002B69013C3370013613685B1A032BEED9FA
:104630000124EEE76008FF1F002370B50468150031
:10464000E366616007F0ECFA0123E366256107F099
:1046500027FB8020064A80001168636B034205D166
:1046600013685B1A032BF8D9012070BD0020FCE70A
:104670006008FF1F70B51D00002304681600E36684
:10468000616007F0CDFA0123E36626610F33626BA8
:104690001A42FCD02B0A23611023626B1A42FCD011
:1046A000EDB2256107F0FCFA8020074A800011680E
:1046B000636B034205D113685B1A032BF8D9012001
:1046C00070BD0020FCE7C0466008FF1F70B51E00EB
:1046D000002305681400EB66696007F0A1FA012366
:1046E000A619EB660F33B4420ED107F0D9FA802039
:1046F0000A4A800011686B6B03420CD113685B1A85
:10470000032BF8D9012070BD21782961696B19420A
:10471000FCD00134E7E70020F5E7C0466008FF1F42
:1047200010B5084CE368002B08D1074B1B685B04ED
:104730005B0C0A336360054B1B68236007F040FA8B
:10474000A06010BDB064FF1FC8F00040CCF0004076
:1047500010B507F065FA0F4B996A9A6A8A42FBD145
:104760000D4C6268A0688A18121A531E884200D342
:104770001300A1602168DA0B52185B0407495B0C37
:10478000636022600B60064B1A6007F089FA2068AC
:1047900010BDC04600F00040B064FF1FC8F00040EC
:1047A000CCF0004070B51F4C23793F2B01D93F233B
:1047B00023711D4B22791A701878C0B207F028FBBC
:1047C00018231A491A4A0B801A4913800B80538008
:1047D000A379194980200B800C21938001334B432E
:1047E000164D191C0001834200D9011C2980D1807B
:1047F0006379002B11D101336371237A012B01D826
:10480000022323726279237A0D4853430A215843C5
:1048100007F02EFB0B4D286070BDA02BEDD9A02317
:10482000EAE7C046A464FF1F480AFF1FD644FF1FE3
:10483000B046FF1FD444FF1FD244FF1FD044FF1FC8
:10484000710200009464FF1FF8B513210020FEF7E9
:10485000C5FD114C011E114D09D10C22104BC1CBCD
:10486000C1C4280007F054F9FFF79CFFF8BD0C22E3
:1048700020000C49FEF786FD0C2802D0084B43CBE4
:1048800043C40C2228000849FEF77CFD0C28EBD01D
:104890000C220021E5E7C046A464FF1F7064FF1FDF
:1048A000ACBF0011FC0C0000F50C0000F0B51D4C75
:1048B0008022A5440400882069465201400507F083
:1048C00047FA902212016A441300200032C832C312
:1048D00016C816C38023144C144FA6689B03334399
:1048E000A3603B6007F034F98823A0685B05C0181B
:1048F00007F016FA0025882329008022A0685B05AE
:10490000C01840196944520007F012FA802301359B
:10491000FF355B019D42EED1A6603E60044B9D4495
:10492000F0BDC046FCEFFFFF2046FF1F9808FF1FA9
:1049300004100000F0B5040087B0002825D06846B8
:1049400007F026FA1B4C022806D1062269462000F1
:1049500006F06EFF002816D06946002301250F26B9
:104960002F00E25C013310091030874038002F001F
:10497000324097403A0002434A610439062BEFD196
:104980006846FFF793FF07B0F0BD182269460A4852
:1049900007F0DEF96A46A300D358013305D0182288
:1049A000FF21684607F0B4F8EAE70134062CF1D19C
:1049B000E9E7C0466509FF1F00090011F0B50025B1
:1049C00004000E0085B0AA4200D186E04B1C087896
:1049D00001934B788978377909021943F3783F06B8
:1049E0001B040B431F43039720706570252800D1DB
:1049F00096E033D8112813D806F03AFF6900220157
:104A0000220122012201AA00B800B10022012201E4
:104A1000220122012201220122012201FC001C01AB
:104A2000232800D1D5E0DB2800D02BE1042A00D8D0
:104A3000ACE01025052A05D0551F2A003800711D4D
:104A400007F0A6F805223100200007F0A1F82A009F
:104A50003900601D07F09CF805353EE0562859D016
:104A600010D8332800D19DE0552839D02628DAD136
:104A70009A4B2900132218001D0007F049F8FEF791
:104A8000BFFA5CE0712800D177E0722800D180E0A5
:104A9000602800D18BE0DC28C5D1022A00D875E05F
:104AA0007378BFB26370B378A370032A05D0033A5A
:104AB000390092B2F01CFEF79FFB10223900E01C77
:104AC000FEF760FCC51C002807DA60705CE00C2271
:104AD0002000834907F05CF80C25280005B0F0BDE4
:104AE000013A804D0C2A13D8002A0AD028000199D7
:104AF00007F04EF8FFF756FE0C2228007A49FEF721
:104B00007BFB29000C22601C07F042F80D25E4E72E
:104B10000C22EBE7734D754B2A0043CB43C2E9E708
:104B2000013A6E4D0C2A11D8002A08D001992800AC
:104B300007F02EF80C2228006D49FEF75DFB2900D6
:104B40001322601C07F024F81425C6E70C22EDE7B9
:104B500005226849601C07F01BF80625BDE71222F4
:104B60006549601C07F014F81325B6E7082263496D
:104B7000601C07F00DF80925AFE77178F72905D813
:104B80005F4B188801F0BAFD0225A6E7FF2363708A
:104B9000FAE75C4B012A03D072785A706270F3E72F
:104BA0005B78F4E72000FFF7F7FA050095E7013A94
:104BB000554D082A0BD8002A05D00199280006F087
:104BC000E7FF01F071F808222900601CD1E70822F4
:104BD000F3E7042A04D94D4D2F6006F0F1FFA860D9
:104BE000FFF7B6FD0422039003A9601C06F0D0FF76
:104BF000052572E7464D062A15D906222800019997
:104C000006F016FE00280ED006220199280006F0B4
:104C1000BFFF06223F492800FEF7EEFA0123394A7A
:104C200051780B43537029000622601C06F0B0FF38
:104C3000072552E7012AA9D07078FFF77BFEA3E78A
:104C4000012800D0EFE6931E334F1A2B04D8737857
:104C5000002B09D100F014F9304B39001D78601C8D
:104C60006A1E06F095FF38E7551E2A0001993800A4
:104C700006F08EFF2A49AAB23800FEF7BDFA00F00E
:104C800035F9E9E7DA281DD1042A00D87EE7082A99
:104C900015D9B37972791B021343F27912041A43BE
:104CA000337A1B0613433B603B680522310020002A
:104CB000039306F06DFF0422601D03A959E7FE234C
:104CC0006370F1E7DE2800D060E7511E012A01D1B0
:104CD000002502E7019800F0CDFFF9E77064FF1F9F
:104CE000B8BF0011A464FF1FFC0C0000ACBF001192
:104CF000F50C00007C64FF1F5C64FF1F2446FF1F4F
:104D0000D844FF1FA064FF1F7545FF1FB064FF1F3D
:104D10006509FF1FADAC0000A166FF1F9F66FF1F66
:104D2000AEDE000070477047020010B5094B0A3232
:104D3000094C92B2DA815A8298811882207802F066
:104D400043FB0422054B012120781A7006F0B8FDC0
:104D500010BDC046AE45FF1FEA66FF1FE966FF1F94
:104D6000013870B5042809D806F0A2FD0309280807
:104D70001200234B0221187806F0A2FD70BD204BD3
:104D80000821187806F07CFF00221E4B1A72F5E706
:104D9000802200241B4B1A4D52001A8108211A68E8
:104DA0002878DC7206F05CFE2100287806F0E8FF27
:104DB000012000F065FE00F077FFDFE7104B0821CF
:104DC000187806F05DFF1048FFF778F80F4B104A8F
:104DD0009B79002093800F4A13808022094B520058
:104DE000D8721A8100F04CFE00F05EFF0A4B5B782F
:104DF000002BC3D0094A136006F072FFBEE7C0461D
:104E0000C064FF1F9464FF1FE144FF1FA464FF1FE1
:104E1000B046FF1FD244FF1FA064FF1F34F00040C4
:104E200010B501290BD1022809D1054B1B78002BA5
:104E300005D02622034B04485A72FFF775FF10BDB8
:104E4000C266FF1F9464FF1FC40900000300F0B591
:104E50000A4D8E18B14202D152008018F0BD0C7874
:104E60002F6824093C5D0F271C700C7801313C40F1
:104E70002F683C5D5C700233ECE7C046CC44FF1FFA
:104E80000D22114B10B51A700C23104C10492370D1
:104E9000093A033B0F48637006F07AFE2D23012286
:104EA0000D490E48A371FFF7D1FF01220C49FFF70E
:104EB000CDFF01220B49FFF7C9FF00220A4910006C
:104EC000FEF79AF910BDC046BE66FF1F9F66FF1F22
:104ED0006BBF0011A166FF1F6709FF1FA666FF1FBA
:104EE0006609FF1F6509FF1FAEDE000070B5124C9A
:104EF000132220001149FEF745FA114D002817DD55
:104F0000AB78002B14D0431C2B7009236B7000234B
:104F100000190370287829000130C0B206F0E8FCBF
:104F2000297822000139C9B2002005F0E9FD70BDE1
:104F3000FFF7A6FFEEE7C046A166FF1FAEDE00004A
:104F40009F66FF1F10B5114B1A781870002A0ED0FB
:104F500000280BD10E4B1A78062A07D85423D340C9
:104F6000DB0703D50B4B187802F02EFA10BD002892
:104F7000FCD0074B1B78012B02D0033B022BF5D84A
:104F8000044B0121187806F09BFCEFE7C266FF1F77
:104F9000E966FF1FEA66FF1F70B54A4E4A4A4B4951
:104FA0003070022005F038FC00F0E8FEFEF728F82B
:104FB00006F0BEFD032246494648FFF747FF2D2471
:104FC000030004221C7044490130FFF73FFF3023E7
:104FD0000470424D424C437083702E3B06222000E9
:104FE0004049EB87FEF7CEF9062813D0200006F0E3
:104FF000CFFE022809D00321200006F091FC8D236A
:10500000E3706E3B2371193363710622200035492A
:10501000FEF7F2F8344B1B68FC335C64FFF766FF65
:105020000020FFF78FFF314C314A0121314B1278BC
:10503000207802F08BF9304A304B1278002120782A
:1050400002F084F901222E4B1A702E4B9B78552BBF
:1050500031D12D4B3B325A722C4B2D4AAB81EA8118
:105060002B826A822021307806F09AFC012040428F
:1050700005F092FD0120404205F02EFEFFF73CF9BD
:10508000FEF700FF00F0A6FC01204042FEF7C6FF3D
:10509000012006F0F5FBF72001F014FB0121307828
:1050A00006F00EFC307802F0EBFA1A4806F088FEA3
:1050B000FEF7F4FD70BD6422174B5B7953431A0071
:1050C0000A32CBE7C064FF1F254D0011214E0011AD
:1050D0002446FF1F5C64FF1F7C64FF1FAE45FF1F5B
:1050E0006509FF1FADAC00004867FF1FEA66FF1FA0
:1050F0000045FF1FE144FF1FBE66FF1F9F66FF1FA5
:105100009066FF1FA064FF1F9464FF1FC409000086
:10511000CE090000C264FF1FA464FF1FF8B50A0097
:1051200020230D001A40194257D0574B1B78002BF3
:1051300050D0FFF70DFB554B554C564E99686268A1
:10514000737A8A1ADB039A4202D36160FEF7A6FDE6
:10515000327A217A531EDBB2994205D1FFF784F9E6
:10516000002000F0DDFD0FE09142F9D3002323720F
:10517000FFF7A4F9012000F0D3FD474F3800FEF7F8
:105180009DFE390006F03CFE637A002B1FD0013BE8
:10519000DBB26372002B1AD1404B9B78552B01D1A7
:1051A00006F09EFDE37A002B0CD000233C4A3A4FD8
:1051B000E3721388380001331380FEF77FFE390055
:1051C00006F01EFE642370795843FFF7ADFD237A85
:1051D0000133237220206840F8BD0BB2002B0ADA9D
:1051E000304B187806F024FD002801D006F010FCA2
:1051F00080200002EFE70224214206D0244B012048
:105200001A72FFF79FFE2000E5E70B071ED5FFF798
:105210009FFA1E4B1E491F4C98684A68637A821A8F
:10522000DB039A4202D34860FEF738FDFFF746F9E8
:10523000FFF71AF9012000F073FD00F0E5FB236889
:10524000DB0701D5FEF7E2FF0820C4E71024214266
:1052500006D00D4B1B78002BD5D1FEF727FED2E7E9
:105260000124214207D0104800F06CF806F078FBCA
:1052700000F036FDC7E70424080020402142ABD0EF
:10528000FEF7E8FEBFE7C046C266FF1FB064FF1F1F
:105290009464FF1FA464FF1FE144FF1FA064FF1F6D
:1052A0008864FF1FC064FF1FC444FF1FF0B51B4B81
:1052B0001B4F1B883A8804001A4E1B4D85B09A423A
:1052C0000DD832889A420AD3184B1A882B889A42F2
:1052D00005D1174A174B12881B889A421BD005200C
:1052E00001F046FA3B8802AA13803388019053806C
:1052F0002B88114D93800F4B02A91B88D3800F4B35
:105300002A78188802F062FF0D4B08212878019A4C
:105310001C7006F0F5FB05B0F0BDC0468E66FF1FA1
:10532000D644FF1FD444FF1FD244FF1F8C66FF1FCB
:105330008A66FF1FD044FF1FEA66FF1FD844FF1F85
:105340008866FF1F13B50C4B1C78002C11D1002868
:1053500001D00A4B18600A4A0A4B11780A4A1078A1
:105360000A4A01920A4A0092002205F0C1FA20007E
:1053700016BD1124FBE7C046E966FF1F8466FF1FC8
:10538000E866FF1FD866FF1FEA66FF1FC466FF1F9F
:10539000C866FF1F10B5064B12201B78052B06D1DF
:1053A000044B13221988044B187801F0BDFB10BD83
:1053B000E966FF1FD844FF1FEA66FF1F10B50024EF
:1053C0000122114B52421870104B1C70104B1A8066
:1053D00002F056F904220F4B21001A700E480C32CD
:1053E00006F026FB102221000C4806F021FB0722C4
:1053F0000B4B1C600B4B1C700B4B1C700B4B1A7037
:105400000B4B1C7010BDC046EA66FF1FE966FF1F0C
:10541000D844FF1FE866FF1FD866FF1FC866FF1F3E
:10542000C466FF1F9E66FF1F9D66FF1FDA44FF1FB5
:105430009C66FF1FF8B5174C0600257806A81424B3
:105440000078052D23D1B41F134FA5B21824BD42F7
:105450001DD88D1FADB2BD4219D8FA256D00AA42E4
:1054600015D21D000D4F0A3DADB2BD420FD80C4CF8
:1054700026800C4C21800C4900240A800B4A1380A2
:10548000FFF714FF0A4B0421187806F0F9FB2000FF
:10549000F8BDC046E966FF1F790C0000750C0000DE
:1054A000D644FF1FD444FF1FD244FF1FD044FF1F28
:1054B000EA66FF1FF0B50BB20D0089B0002B00DBD0
:1054C00070E1A44E307806F0B3FB041E50D0037890
:1054D000A22B00D122E1D02B1AD0912B45D14378B9
:1054E0000E2B42D19C4B82889A423ED19B4A8368C4
:1054F0001278052A39D1032018567F2835D0984BC9
:105500001B68002B31D05B68002B2ED098472CE015
:105510008078072829D806F0CBF90428183F3F7473
:10552000A8D86378002B0CD101218C4B19708D4BBE
:105530001A78002A5BD08C4B307801F007FF0028E6
:1055400055D00722854B1A7051E061780029F8D1B7
:10555000E378002B11D0854A854B1278307801F022
:10556000F5FE60706378002BEBD1200006F050FA56
:1055700080200002684009B0F0BD784B1B78022BF8
:10558000F3D00121307806F04BF90028EAD101214F
:10559000307806F095F9E5E76378002BD1D16F4FAD
:1055A000032807D13B78052B02D101333B701EE065
:1055B0000223FBE76F4B1A886F4B0293002A0BD034
:1055C0001B78002B03D00121307806F099FA3B7844
:1055D000062B04D1013BE9E7029B1A70F7E7042B85
:1055E00041D10121029B3078197006F069F95C4BBA
:1055F0001B68002BB9D01B68002BB6D0574A107817
:1056000084E76378554F002B27D10622211D5B4884
:1056100006F0BEFA62895A4B5A491A80A2895A4B3F
:105620001A80E3890B800521397058490A80584A4D
:105630001380228A574B1A80574B1B78012B09D1B4
:105640001F2001F095F8FA2292004243042130789D
:1056500006F056FA0022484B75E7312B00D070E770
:105660000022454B1A700323A0E70622002143487D
:1056700006F0DEF90023454A04211380444A3078BD
:105680001380444A138006F0FBFA0821307806F0B4
:10569000F7FAA379083B5A425341304A0333137057
:1056A000304B1B78002B06D0334B30781A78002A09
:1056B00006D001F089FE0122314B52421A8096E752
:1056C0000121197006F0FCF8F5E70821307806F0A2
:1056D000D7FA6378002B00D047E72C4B2D4F02936D
:1056E000E388029A04211380294B3078039323899D
:1056F000039A138063893B8006F092F8002800D05B
:1057000033E7264B1B68002B00D12EE70399029844
:105710003A88098800881B68984726E74379132B45
:1057200000D022E70389012B0AD11D4B1B78022BE5
:1057300006D10821307806F0A3FAFFF72BFE14E714
:10574000052001F015F808210200307806F0D8F99C
:105750000BE7C046EA66FF1F05140000E966FF1F5D
:105760008466FF1F0045FF1FE144FF1FBE66FF1F49
:105770009F66FF1FC066FF1FC266FF1F9166FF1F67
:10578000D844FF1F9866FF1F9A66FF1F8E66FF1F93
:105790008C66FF1F8A66FF1F9066FF1F8066FF1FD3
:1057A0008866FF1F8020C001014200D0E2E6CB07DF
:1057B00031D5324B1B78002B1DD0314E05AC3378E0
:1057C000052B1AD1023B23702E4B21001B7823722C
:1057D0002D4B1B7863722D4B187801F05BFD002870
:1057E00009D007202A4B30701B68002B03D01B68A0
:1057F000002B00D098470120BCE60E20254B062246
:105800001B7825492370254B1B78637002ABC018A9
:1058100006F0BEF9D8E7022308001840194209D063
:10582000174B1B78052B03D11D4B188806F0A8F9E0
:1058300002209FE60424214203D0FFF737FD200019
:1058400098E6082308001840194200D193E6154B4A
:105850001C78012C03D0022C0DD008208AE6124BB4
:10586000124A134913481B8812880988008800943B
:10587000FFF7E0FDF1E7FFF78DFDEEE7C266FF1FE2
:10588000E966FF1FDA44FF1F9C66FF1FEA66FF1FE1
:105890008466FF1F9E66FF1FDB44FF1F9D66FF1F80
:1058A000D844FF1F8866FF1FD044FF1FD244FF1F4C
:1058B000D444FF1FD644FF1F10B502A804880B2054
:1058C000002C10D1496808784978090201430C4836
:1058D000814209D1022119800A4B59881170DB7865
:1058E00000205BB2537010BD074C0A20A142FAD1D0
:1058F00002211980034B998811705B79F0E7C0464B
:105900006E2A00008864FF1F6F2A0000F7B515009B
:1059100008AA16884A680F4F147852781202224358
:105920000A24BA4214D10122DBB2019200962A0065
:1059300005F0E4FE041E0BD1074B1B68002B07D0BB
:1059400068782A780002104342425041013098475B
:105950002000FEBD02290000FC66FF1F30B50125B6
:1059600003790400BFB02B4227D01549408805F0C9
:1059700031FA28420DD06A46124B69465B8D13807E
:1059800002235380104B5B8893806088002202F0D2
:1059900013FB0E49608805F01DFAC0070DD56A4655
:1059A0000B4B69461B88138002235380064B9B8850
:1059B00093806088002202F0FFFA3FB030BDC046FD
:1059C000F466FF1F0445FF1F8864FF1FEC66FF1F7E
:1059D0005E45FF1F10B5074C0749200005F0B0F9E0
:1059E0002000064905F0ACF90721054A054805F0F5
:1059F00069F910BDFFFF0000F466FF1FEC66FF1F92
:105A000038C000110445FF1F10B5024803F056F9D5
:105A100010BDC0465D590011082110B50E240A4A78
:105A2000C307DB170B405179A1430B43537102238A
:105A3000184202D051790B4353710423184202D00B
:105A400051790B43537110BD7545FF1F0A2110B5E5
:105A50000F240A4AC307DB170B401178A1430B43FD
:105A60001370830703D5062311780B431370400787
:105A700003D5012311780B43137010BD7545FF1F2B
:105A800010B5054B102419780A00A243002801D054
:105A900022000A431A7010BD7545FF1F662110B51C
:105AA0002024134BDA788A431979DA70A143241938
:105AB0000C431C71542812D9602001431971042130
:105AC0000A43DA700222D9780A43DA702022D978A0
:105AD0000A43DA704022D9780A43DA7007E0442892
:105AE000EDD83428EED82428F0D81428F2D810BDE8
:105AF0007545FF1FF8B50E23384C050062792679ED
:105B00001A4011339E43364B62712671984204DD70
:105B10006E23E3716C3BA371F8BD324B984203DAFC
:105B20001A23E3711C33F6E700232F49A371E371B5
:105B300083B259182D4889B2814224D9681D0A219F
:105B400000B206F095F92A4B00B29D4244DC0500F4
:105B50006421280006F08CF90A2100B206F020F931
:105B6000244F09B2E2797B5C1343E3710A212800D8
:105B700006F07EF90A2100B206F012F91D4F09B2B3
:105B80007B5CA2790EE001210A436271002D1CDAD0
:105B90005B421DB20423A371A379632DD8DCFA22E2
:105BA000092DE3DC1343A3710A21280006F0F8F85D
:105BB0000F22114F09B27B5C1A4016431F229343F8
:105BC0006279267113436371A6E7FA239B009D4215
:105BD000E2DB0123E371BBE70500FAE77545FF1F30
:105BE0001B4E00001DFCFFFFCB070000960F0000BE
:105BF0000A27000082C0001172C0001170B51B4D51
:105C000004002B7900290DD0802213432B71632CC3
:105C10000BDD76236A7813436B704023AA78134315
:105C2000AB7070BD7F221340F0E72300093306DA22
:105C300058236A7813436B70AA786C23EFE70C4EF5
:105C4000002C0ADA2023644224B26B700A2120005F
:105C500006F0A6F809B2735CE2E7092CF6DD0A212A
:105C6000200006F005F900B2335CEEE77545FF1F32
:105C700062C00011F8B50A4F05003B780E00002BFA
:105C80000CD0084C2000FEF72DFC33002A00200029
:105C90003978FEF71BFD2000FEF762FCF8BDC04618
:105CA0000967FF1F8045FF1F70B50A4E0A4D082285
:105CB0003100280005F0BCFD002809D0074C310058
:105CC0000822280005F064FF09212000FFF7D2FF19
:105CD00070BDC0467545FF1F0167FF1F0067FF1FAE
:105CE000102110B50D4B1A780A401A70DA78563127
:105CF0000A40DA70602219791140223ADA71083AC2
:105D00009A71AA325A71DF3A0A431A7106225A70FE
:105D100029329A70FFF7C8FF10BDC0467545FF1FB6
:105D200010B5002824D0134C0A210223E05E06F0AF
:105D30009FF800B2FFF7DEFE0423E05E642106F068
:105D400097F8012100B2FFF759FF207AFFF7A6FE6E
:105D50000320FFF761FE0020FFF778FE064B18785E
:105D6000053843425841C0B2FFF78AFEFFF79CFF57
:105D700010BDC0468864FF1FE966FF1F70B500258F
:105D80000A4C2000A571FEF7ADFB10233E21200038
:105D9000074AFEF79BFCA84200D13E35054B200088
:105DA0001D70FEF7DDFB0123A37170BD8045FF1F51
:105DB00052C000110967FF1F0200F0B501270A4811
:105DC0000A4E51188B1A002B00DCF0BD0824157800
:105DD0004308684038404000805B013C58406D08F3
:105DE000002CF5D10132EDE7FFFF000092C0001159
:105DF000F0B500250F269D4200DBF0BD4C5D070984
:105E000044403440A400A05801357840F3E7000036
:105E1000F0B589B06A460D000B000F271100103550
:105E20001C780133260024093E401670547002325B
:105E3000AB42F5D12023024AFFF7DAFF09B0F0BDEB
:105E400098C00011F0B54E780B7889B036020C007E
:105E5000170001901E43012A61D9954B9E4200D83C
:105E600077E001339E421CD1062A17D1CA788B787D
:105E700012021A430B791B0413434A7912061A4380
:105E80008C4B5A6100221A705A808B4A5A608B4A96
:105E90009A608B4ADA60002009B0F0BD8822520572
:105EA000EEE7884B9E423CD182498B78002B00D094
:105EB000F6E00C2A31D10F22A3789343E278120244
:105EC00013432279120413436279120613434B6081
:105ED000E279A07912020243207A00041043627A28
:105EE00012060243CA60E27AA07A1202024376489E
:105EF0004A81834208D804236E49142201980B700A
:105F000005F046FE1420C7E71201D21889235B056D
:105F10009A42F0D801238B70BDE7022AFAD00523FC
:105F2000EAE76A4A01239642E6D1FFF733FA052FE2
:105F30000CD9E378A2781B021343227912041A4386
:105F400063791B061343624A0393136005F0C8FE8E
:105F5000A1E7584D2B78002B9DD1AB78002B00D1B9
:105F6000A0E02B8901339BB20093B34200D091E0B3
:105F7000132AD4D9CF7C8B7C3F02122120001F43EF
:105F8000FFF71AFF874200D08EE0002E3DD1E37864
:105F9000A2781B0213432279E96812041A43637939
:105FA0001B06134303930A228B4212D1FF23A370D3
:105FB000E370237163716B89002B09D1E37B227C31
:105FC0001B0212041343A27B13431B0901336B8191
:105FD00000226B89002B8ED0002A67D168683701B8
:105FE0003818000B6B6900030390984205D968616B
:105FF00005F096FEEB780133EB7068681022A11C67
:10600000381805F095FE2E8145E76F89009A7B1EB2
:106010009BB293423AD1E278A37812021A432379D1
:1060200005A81B04134362796C6812061A43EB68D7
:1060300000920392211D0C22049305F0A9FD01207A
:10604000260004A940421036FFF7E2FE013F012F6F
:1060500017D1009A0B232861824200D04CE704221A
:106060001C49200005F064FE042203A9686805F0BD
:106070006FFEE968039AFF23914200D13CE7F73BAA
:106080003AE73100FFF7C4FE1036DFE70923B742D5
:10609000A4D831E7009BB34200D9FCE607232BE7E5
:1060A000022329E7032327E7062325E70A2323E71B
:1060B000FFFE00008845FF1F00000111FFFF0000E8
:1060C0005048593601FF0000FFFF001102FF000099
:1060D00034F000409445FF1F10B5034C0B00012223
:1060E000210000F06BFA10BD996200110B8870B5A9
:1060F00006000D000224162B11D92B00032209499A
:1061000000F05CFA041E0AD1074B2A881B88191C70
:10611000934200D9111C300089B200F0EFFA200040
:1061200070BDC046C56200116267FF1F10B54A7896
:106130000400013A0B000220012A07D80A78002A3D
:1061400004D005222000024900F038FA10BDC046F4
:10615000F36200110A7810B50B0004000220002A37
:1061600004D007222000024900F028FA10BDC046E2
:106170009F6300110A7810B50B0004000220002A6A
:1061800004D009222000024900F018FA10BDC046D0
:106190000564001110B5034C0B000B22210000F028
:1061A0000DFA10BD3564001110B5034C0B000D2223
:1061B000210000F003FA10BDA764001110B5034CD4
:1061C0000B000F22210000F0F9F910BD016500114C
:1061D0000A7810B50B0004000220002A04D0112216
:1061E0002000024900F0EAF910BDC0461165001117
:1061F000002310B51322190000F0E0F910BD0000D3
:1062000010B5034C0B001722210000F0D7F910BD88
:1062100063650011002310B51922190000F0CEF9B2
:1062200010BD000010B5034C0B001B22210000F034
:10623000C5F910BD9D650011F7B584890D000600F4
:106240000121002C22D000238268D3561778002B1E
:106250001EDA0C2C1AD90C3CA4B2131940880093F6
:10626000230002F086FE431E984101307B06DB0FBF
:106270006B703F23013C1F40A4B22870AF70AC800C
:10628000002C07D0B3680133AB6000210800FEBDCD
:106290000020EBE7AC60F8E70B7803704B884370A5
:1062A0004B881B0A83700B79C3700420704704204D
:1062B000022B06D10020537811781B02009A0B4361
:1062C000138070470B8803700B881B0A43700220F1
:1062D00070470420009983420AD1537810781B023A
:1062E00003430B80D37890781B02034300204B803C
:1062F0007047F8B50D004B7801240021461C03704F
:106300002B788B4201D82000F8BD6B78B01C4F1C55
:10631000012B10D1890069184B88022233704B88F9
:10632000B9001B0A7370691805F07AFD043604344D
:10633000A4B2F9B2E4E7122359436B185A88043126
:1063400032705B8810221B0A7370691805F068FDB3
:1063500012361234ECE770B5049D14001E00052BB4
:1063600001D8042070BD637812781B0213432B8080
:10637000E378A2781B02134302226B802A71211D4D
:10638000681D063E05F04CFDB2B22A81F02AE8D81D
:106390002800A11D0A3005F043FD0020E2E700239C
:1063A00010B50A789A4201D8900010BD9A008A1858
:1063B0005488013304705488DBB2240A44709488F2
:1063C00084709288120AC2700430EAE710B5110096
:1063D000029C062B04D004201022142B01D010BDE7
:1063E000022222714B7808781B0203432380CB786A
:1063F00088781B02034363800431601D05F010FDA3
:106400000020ECE710B50C788B7804315C43E4B2E3
:1064100003702200013005F003FD601C10BD042054
:10642000022B06D10020537811781B02009A0B43EF
:106430001380704710B50C000A88023105F0F0FC9B
:10644000208810BD70B504000D0004981100012BC8
:1064500001D8042070BD16785278120232430280AF
:106460000200F83255701470E825002C00D10C356C
:10647000023B9AB24280AA42EBD80231043005F0C6
:10648000CFFC0020E6E70420009983420AD153782C
:1064900010781B0203430B80D37890781B020343D0
:1064A00000204B80704710B50C000A88023105F0BF
:1064B000B7FC208810BD000070B501211E0004202B
:1064C000049C0E400B4218D1CB40DDB28D4214D952
:1064D0000A49DBB2098899420FD32300F6331D70B5
:1064E0003300580011184978165C09023143013312
:1064F0002152D9B28D42F4D8002070BDA845FF1FAB
:1065000010B50C000A88023105F08AFC208810BD05
:1065100010B50C788B7804315C43E4B20370220030
:10652000013005F07DFC601C10BD10B51100029813
:10653000032B01D8042010BD14785278043B1202BA
:1065400022430280CA788C781202224342809AB297
:106550008280F22AEED80431063005F061FC00207A
:10656000E9E710B50C000B8803700B881B0A437019
:106570004B8883704B881B0AC3708A8804300631AD
:1065800005F04EFCA088043080B210BD0420012B21
:1065900003D100201378009A1370704710B50C00D7
:1065A0000B8803700B881B0A43704A880230043141
:1065B00005F036FC6088023080B210BDF0B589B0BD
:1065C00003931E4B029242000700D05A019102F041
:1065D00020F81325061E2DD0029B01240370019B79
:1065E000002B04D0001903999847001984B26B4618
:1065F0001B7A5BB2002B0FDA1021380002F01CFB73
:106600001925002813D130003219E1B202F066FCDE
:10661000051E0CD10C34A4B2042304AA380005A929
:1066200093800696948101F0AFFD051E02D03000E4
:1066300005F0FEFB280009B0F0BDC0466067FF1FF3
:1066400070B505000C0000280CD00020814209D054
:1066500010222000044905F0E3FB01202B7823736E
:106660006B78637370BDC046D8C00011F0B50600EA
:106670000D0017001C0085B002291BD00020102936
:1066800007D1022B07D0102B03D115E00020102CCE
:1066900008D005B0F0BD69463800FFF7D1FF2A00E9
:1066A00069460BE069463000FFF7CAFF22006946E1
:1066B000380004E0022BE9D12A003900300005F04F
:1066C000C7F8E6E7031CF72800D9F7230320084999
:1066D0009AB2013A0B80D317034006499B189B10CE
:1066E0000B80D30F04499B185B100B807047C0468A
:1066F000AC45FF1FAA45FF1FA845FF1F034B1B8882
:106700008B4202D3024B4000C1527047AC45FF1F81
:106710006067FF1F014B4000185A70476067FF1FFA
:106720001722014B1A8070476067FF1F70B5050084
:106730000E2005F065F9041E13D0D023037000234A
:106740000622837007494570033005F069FB064B4C
:106750002100DA8A62811B7E2373044B187805F0CE
:106760001FFA70BD7C67FF1F6C67FF1FFC45FF1F92
:10677000262803D8024B4000C05A70470148FCE766
:10678000AE45FF1FFFFF000070B506000C00094D6D
:106790001C220021280005F04BF9074B1E70074B07
:1067A0001C7005F025FB0123002801D000231220D6
:1067B0002B7070BD6C67FF1FFC45FF1F8D67FF1FAF
:1067C00070B505000D4C0800E260A16010220021A8
:1067D000656005F075FA012803D11021A06802F068
:1067E00058FD10220021280005F06AFA012803D183
:1067F0001021606802F04DFD70BDC0466C67FF1F40
:1068000070B5041E05D1002903D006220D4805F0FD
:1068100007FB0D4B1D78012D11D1002C05D1022253
:106820001A7005F0DDF8280070BD00221A70074BC1
:106830001B78FF2BF7D02000FFF778FFF3E7002548
:10684000F1E7C0467C67FF1F6C67FF1FFC45FF1F19
:10685000030010B5002801D1002010BD00780B4ABC
:10686000002803D15988D1821B7913761378022B23
:10687000F2D10023984200D103331370044B1B78EC
:10688000FF2B01D0FFF752FF0120E6E76C67FF1FE7
:10689000FC45FF1F002911D000280CD04B7901289E
:1068A00003D140225242134303E03F221340032806
:1068B00002D001204B7170474022F4E70800FAE74C
:1068C00070B5094D0100287800280BD0074C06222E
:1068D000200005F0A5FA21002878FFF7DBFF200053
:1068E00005F01EF970BDC0468C67FF1F6667FF1F6D
:1068F00000290AD0012808D13F224B799343C02BAD
:1069000003D0403B5A425341981C704770B5174D15
:1069100006002B78FF2B15D00A2005F071F8041E15
:1069200010D0D0230370C83B8370114B11491B78E2
:106930004670C3700622043005F072FA21002878F0
:1069400005F02EF90C4B1B78012B0DD10B4B1B685E
:10695000002B03D09B68002B00D09847084B0421E4
:106960001878084A05F07CF870BDC046FC45FF1F4A
:106970008C67FF1F6667FF1F8867FF1FB467FF1FD5
:10698000B867FF1F60EA0000014B98687047C04677
:106990006C67FF1F014BDB68186870476C67FF1F4F
:1069A000074B10B5DA68136801331360054B18788C
:1069B000FF2803D08021C90104F082FF10BDC0462A
:1069C0006C67FF1FFC45FF1FF7B50E0002F0C8F80B
:1069D000051E1CD00E4B06621F78002F00D10778D1
:1069E000AB791020019305F00BF8041E0FD0D023D3
:1069F0000380C73B8370019BE91DC37006220430EE
:106A000005F00EFA21003800E66005F0C9F8F7BD80
:106A1000FA45FF1F014B18787047C0468C67FF1F6F
:106A2000054B002805D1054B1A78054B002A00D1EB
:106A3000014B18007047C0467C67FF1F8C67FF1F23
:106A40006667FF1F014B58687047C0466C67FF1FA1
:106A5000024B1868431E9841C0B270479067FF1FF1
:106A6000421E03000120152A03D9FF3B5A4253411D
:106A7000D8B27047F0B51C0000230E0085B003901B
:106A800002920B70029A934201D3002019E0E55C58
:106A90005A1CD2B2002DF8D0029851198142F4DC70
:106AA0000233DFB2A35C18000193FFF7D9FF00287F
:106AB00007D0013D019A0399EBB233708A4202D1AB
:106AC000E01905B0F0BDDB19DBB2DBE710B50C0057
:106AD00002F09EF803001220002B03D021005888FA
:106AE00004F06EFF10BD000070B50E4D84006359B8
:106AF000002B15D0186A002801D004F0E9FE2B59AC
:106B0000586A002801D004F0E3FE2B59986A002847
:106B100001D004F0DDFE285904F0DAFE00232B51E9
:106B200070BDC0469C67FF1F1C4B70B504000E0073
:106B3000150099420AD11A4B1B68002B01D1122073
:106B400070BD1B68002BFAD09847F9E7154B9942A6
:106B500015D1134B1B68002B0AD01B68002B07D0E4
:106B60009847002804D1104B1C70104B1D70E7E7AC
:106B700029002000FFF7AAFF0028E1D1F3E7080071
:106B800001F0EEFF0028DAD003780320A342D7D12A
:106B90002900300004F014FFD2E7C046FEFF0000D9
:106BA0009867FF1FFFFF00009567FF1F9467FF1F97
:106BB000F7B50400808801F0D3FF0025A84203D078
:106BC0000578A08802F008F81C4E3378002B1FD0FF
:106BD000AB421DD11A4B28001978FFF777FF002828
:106BE00018D000233370A3790820A778A6880193D2
:106BF00004F006FF011E0DD0D0230370CA3B837042
:106C0000019B477086808371280004F0C9FF01E072
:106C1000002DE8D1A0880B4B8200D358002B01D067
:106C2000FFF762FF1721A088FFF768FDA08801F039
:106C300027FDA08801F0FEFDF7BDC0469567FF1F48
:106C40009467FF1F9C67FF1FF0B587B01D000CAB5A
:106C50001B88070001930DAB1B88142002930EAB19
:106C60001B88160003930FAB1B880091049310AB95
:106C70001B88059304F0C4FE041E1AD0D0230370B1
:106C8000CB3B47708370C670062229000430002D6C
:106C900011D005F0C5F8019B21006381029B00988B
:106CA000A381039BE381049B2382059BA37404F0CF
:106CB00077FF07B0F0BD04F0BBFEECE7F7B500933B
:106CC00008AB1B8807000C200D001600019304F090
:106CD00097FE041E13D0280001F042FF00280FD0B9
:106CE0000078D0232370C93BA370009B210023812F
:106CF000019B6770A580E680638104F051FFF7BDBA
:106D0000014B1878EDE7C046FC45FF1F13B50400A2
:106D100064890389C2888188C0780094FFF7CEFF18
:106D200013BD000010B5044C2068002803D004F007
:106D3000CFFD0023236010BDA067FF1FA122F0B587
:106D4000818892004A43384B384F1B6804009B18D7
:106D50009D2292009B18827989B01A603B68002BB3
:106D60005FD01D78324B1B68002B04D05B68002B72
:106D700001D000209847260008363100E079FFF75F
:106D8000B7FD237DE0710200E0780493638A290057
:106D90000393238A0293E3890193A388009333002A
:106DA000FFF752FFE378002B0BD1E289A379A1888A
:106DB00002920196E27928000092012201F0DAFEA7
:106DC000E0703B68002B20D0FFF7ACFF194D28780E
:106DD00000281AD0184B1978FFF778FE002814D035
:106DE0002B78E67808200793A78804F009FE011E97
:106DF00009D0D0230370CA3B4670837087808671A8
:106E0000079804F0CDFE00232B701721A088FFF710
:106E100075FCA08801F034FCA08801F00BFD09B0DE
:106E2000F0BD064B9DE7C0463409FF1FA067FF1F5A
:106E3000B467FF1F9567FF1F9467FF1FFC45FF1F87
:106E4000F8B5070008000E0001F08AFE041E18D0F5
:106E50002620FFF78DFC051E00D12578062004F0C2
:106E6000CFFD041E0DD00021062204F0E1FDD02349
:106E70002370C23B21006770A370A680E8B204F0C3
:106E80008FFEF8BDF0B585B001930AAB1B78070003
:106E900002930BAB1B7808000D000092039301F0E6
:106EA0005FFE061E22D0102004F0AAFD041E1DD095
:106EB0001022002104F0BCFD2620FFF759FC002819
:106EC00000D13078D0232370C13BA370009B2100F8
:106ED0002372019B67706372029BA580A372039B60
:106EE000C0B2E3720C9BE36004F05AFE05B0F0BD43
:106EF000F7B50D00019001F033FE071E20D00E20E3
:106F000004F07EFD041E1BD02620FFF731FC061E78
:106F100000D13E78D0232380C53B0622A370F91D03
:106F2000E01C04F07DFF019B2A0063810123DD400A
:106F30001A401D40210022736573F0B204F030FE48
:106F4000F7BD0000F0B585B0029010000D001700ED
:106F50000A9E039301F004FE041E31D0029B002B15
:106F60002ED1039B02795B0724D5122313430422FD
:106F7000002E08D10B99002905D10C99002902D1C6
:106F80000D9900291AD01A430D9B2271002B00D0B5
:106F9000C9E0002E00D1CFE0002D00D0CCE0606A27
:106FA000002801D004F094FC1C21300004F0A0FE65
:106FB000606205E002239A430E33D7E793432371BF
:106FC000654BBA00D458002C00D1AAE0002E10D096
:106FD000236A002B03D11C2004F08AFD20625E4B43
:106FE000BA00D358186A002803D01C22310004F0DC
:106FF00017FF0C9B002B12D0574CBB001D596B6A1E
:10700000002B03D1162004F073FD6862BB00E35827
:10701000586A002803D016220C9904F001FF0D9B3A
:10702000002B11D04C4DBC006659B36A002B03D124
:10703000142004F05DFDB0622B59986A002803D03B
:1070400014220D9904F0ECFE380001F089FD051EB4
:1070500067D0414BBA00D358002B62D01A6A342053
:10706000002A00D11C389A6A002A01D0143080B25C
:107070000B9A002A01D01C3080B25B6A002B01D031
:10708000163080B204F0BCFC041E4AD01822002145
:1070900004F0CEFC2620FFF76BFB0190002801D105
:1070A0002B780193D0232370029B200063700A2366
:1070B000294EA370039BBD00A371AB59A780196A29
:1070C0001830002905D01C22A06004F0A9FE200081
:1070D00034307359996A002907D0030014221433FD
:1070E000E060029304F09CFE02980B9B002B08D0FA
:1070F00003001C221C330B992061029304F090FEC4
:1071000002987359596A002903D01622606104F06D
:1071100087FE6B462100187904F042FD3800FFF726
:10712000E3FC05B0F0BD10220D9B0D991B69A01862
:10713000236204F075FE2CE70B9B002B00D13FE788
:10714000012D00D03CE7606A002801D004F0C0FBAC
:107150001C210B982AE7C0469C67FF1F10B5044C02
:107160002068002803D004F0B3FB0023236010BD87
:107170009067FF1F0B4B07B51A68002A01D100204A
:107180000EBD6946531C012012780731FFF772FCCF
:107190000028F4D002780123100018401A42EED0E3
:1071A000EEE7C046AC67FF1FF0B51F4F01203B68FC
:1071B00087B0002B25D09B78059300F0B3FB002807
:1071C00021D00A20FFF7D4FA04000B20FFF7D0FAF1
:1071D000164B05001E78731E9E413B68F6B2191DC2
:1071E000D878FFF757FB3B682900DA7A043303921B
:1071F0009A7901930292009033002000059A04F0DE
:1072000087FD07B0F0BDFFF7B5FF002805D00620C9
:10721000FFF7AEFA04000720D8E70820FFF7A8FA26
:1072200004000920D2E7C0469067FF1F8C67FF1F4C
:1072300070B50A4E040033780D00FF2B0DD00420EA
:1072400004F0DEFB011E08D0D0230370CE3B457056
:107250008370C470307804F0A3FC70BD0C46FF1F2F
:1072600070B5040006200D0004F0CAFB011E0AD010
:10727000D0230370CD3B8370054B44701B68858021
:10728000187804F08DFC002C01D0FFF767FF70BD6B
:107290009067FF1FF8B5264F06003B680D001124CC
:1072A000002B05D10522234B1B78134202D1122457
:1072B0002000F8BD204A10241268002AF8D0127865
:1072C000002AF5D0DB0719D52B789A1E012A1AD887
:1072D0000C2004F00DFC132438600028E8D00023B3
:1072E0000A22437029000670023004F099FDFFF76E
:1072F0005BFF041E0AD0FFF731FFD9E700F012FB55
:107300000028E1D1E4E7002BE2D0D0E70B4B1B785B
:10731000032BCDD11D20FFF72BFA094B1880002835
:10732000C6D0084B04211878074A04F099FBBFE740
:107330009067FF1F8D67FF1FAC67FF1F8C67FF1FE4
:107340008A67FF1FB867FF1F60EA0000F7B5019367
:10735000194B14001A78052306000F0012201A4258
:1073600021D0012920D1154B1D68002D1BD00220F2
:107370001F2C18D8002C02D0019B002B13D0104BCF
:107380001F221E706E1C0021300004F051FB019979
:107390002200300004F044FD310020002C70002F4A
:1073A00006D004F015FCFEBD064B12201D68DCE77C
:1073B00004F09EFAF7E7C0468D67FF1FAC67FF1F1A
:1073C0000C46FF1FA867FF1FF8B50F4E1224336845
:1073D000002B17D01B780F3C834213D100250B4F95
:1073E0000221387804F04CFC094B042138781D80C8
:1073F00004F046FC074B28001D8033685C7004F0E5
:107400003FFD04002000F8BD9067FF1FB867FF1F15
:10741000A467FF1F8A67FF1F70B5012823D11B4C8B
:107420002388002B03D01A4A1578002D07D0194B5A
:107430001B68002B02D01878FFF7C6FF70BD3B2BEE
:1074400002D93C3B2380F9E7134E0221307804F047
:1074500017FCFA222388920002215A43307804F064
:107460004FFB2580EAE70B4B1B68002BE6D00B4B4C
:107470001B785B07E2D5084B0221187804F000FC6A
:107480000022024B1A80FFF769FED7E7A467FF1FAF
:107490008867FF1F9067FF1FB867FF1F8D67FF1F7B
:1074A000F8B51E4D2868002803D004F011FA002317
:1074B0002B601B4E3068002803D004F009FA00232B
:1074C0003360184F05243B7818002040234221D018
:1074D000154800F02BFA3B78234213D0202004F00B
:1074E00007FB2860002813D02022002104F0A0FA16
:1074F000202004F0FDFA041E306005D02022002177
:1075000004F096FA002004E0286804F0E1F92C6009
:107510001320F8BD00F00AFAF4E7C046AC67FF1F7D
:10752000A867FF1F8D67FF1F0046FF1F10B50A4C9D
:1075300023681A1E0ED0002808D10130587004F0BC
:107540009FFC002805D02368002B02D00021FFF704
:1075500087FE0122100010BD9067FF1FF7B5274E70
:10756000050033680191181E21D05C78244F012C4E
:1075700030D1FFF7FFFD002825D02000FFF7F8F8F5
:107580000400412814D91F4B022118781E4A04F028
:1075900067FA1E4B3C3C1C80022233685A703B78D1
:1075A000002B14D128000199FFF75AFE0120FEBDDF
:1075B000FA2292004243002AEED0124B02211878A0
:1075C00004F09EFAE8E7FFF7D3F80200F3E70023A0
:1075D0003B70EBE73B78002BE8D1032004F010FA76
:1075E000011E08D0D0230370CC3B457083703368F4
:1075F000187804F0D5FAFFF7B1FDD7E79067FF1FC1
:107600008867FF1FB867FF1F60EA0000A467FF1FBD
:1076100010B51749838802008B4220D011D8154934
:107620008B4217D0144900205B1899B2012907D862
:10763000926811785A425341D8B2FFF7F9FD012000
:1076400010BD0E4A00209B1807229BB29A4240416F
:10765000C0B2F5E783681878FFF768FFF0E7836842
:1076600099785A78090218781143FFF777FFE7E70E
:107670000A20000006200000F8DFFFFFAFDFFFFF59
:10768000014B18707047C0460D46FF1F10B5064CE1
:10769000207001F041FA207804F01AFA05212078D0
:1076A00000F062FD10BDC046B867FF1F0BB273B596
:1076B0000D00002B00DBC4E0884B187804F0B8FA0A
:1076C000041E0ED00378912B0FD0A22B00D1A1E085
:1076D000834B1878FF2852D0210004F061FA00286B
:1076E0004DD180200002684076BD43780F2B76D0C4
:1076F00013D8052B70D00E2BEAD18088794B984295
:107700002BD8794B98421BD8784B9842E0D1A3688C
:107710001878591CFFF774F838E03E2BD8D18378DD
:10772000032B74D06CD8012B6ED0022BD0D1704BB0
:107730001B68002B23D05B68002B20D098471EE0ED
:107740006C4BC0180C28C3D804F00AFB1DC2C2152C
:107750000BC20B0B0B3223C23C00674BC01807282F
:10776000B6D8664B1B68002B09D01B68002B06D0CF
:10777000200098470AE0A3681878FFF7C7F82000B0
:1077800004F046F9ADE7A068FFF762F800289FD043
:10779000F5E7A3681B78002BF1D0554B1B68002B35
:1077A000EDD01B68002BEAD0210055489847EDE743
:1077B0004F4B1B68002BE2D01B68002BDFD0210051
:1077C0005048F3E7504B1B68002BD8D05B68002B68
:1077D000D5D021004348E9E7FFF7EAF9CFE78088F1
:1077E0004A4B984203D04A4B984200D070E7464B30
:1077F0001B68002BC3D05B68002BC0D02100D5E7ED
:10780000153B012BBBD963E7FFF798FAB7E7FFF702
:107810007DFAB4E73F4B1B78042B07D100236A465F
:1078200013800179408800F0C5FCA8E7364B1B683F
:10783000002BA4D05B68002BA1D0010036489847EC
:107840009DE7012421420AD0294B1B68002B04D05C
:107850005B68002B01D000209847012043E78B078D
:107860000AD5264B1B68002B04D05B68002B01D087
:1078700020009847022036E70421280008400D42E6
:1078800000D131E7254E3388002B21D0013B9BB23C
:107890003380002B1AD1FFF7DBF800280AD0204BE9
:1078A0001C70164B1B68002B04D05B68002B01D0AA
:1078B00020009847FFF7C6F8694601F001FD6846C9
:1078C000FEF7FEFF1D20FEF753FF308004200AE77D
:1078D000024B187804F0D4F9F8E7C046B867FF1FE8
:1078E0000D46FF1F0E2000000120000009100000BF
:1078F000B067FF1FFEDFFFFFAFDFFFFFB467FF1FB3
:107900000C2000000B2000009867FF1F0D200000D6
:10791000132000008D67FF1FFFFF00008A67FF1F15
:107920008867FF1F10B501F09BF910BD014B18606F
:107930007047C046B467FF1F0B880020162B01D884
:1079400017230420014A13807047C0466267FF1F57
:1079500000207047074A03001188814207D09188B0
:107960000020994202D10130800010187047002099
:10797000FAE7C046C067FF1FF0B58F7806000D001C
:10798000C7B01E2F15D1FFF7E5FF051E03D1002458
:10799000200047B0F0BD00223B003100C0780092CB
:1079A00000F0B2FB0400A81C00F0D3FBFF23EB7037
:1079B000EEE7264B062403931B78FF2BE8D0182F05
:1079C000E6D87B08224A013BDB0002929A58944693
:1079D000002ADDD0029AD3185B68002BD8D0087833
:1079E000002802D14B78012B02D10624122FCFD1CF
:1079F00007AFAB88697800976446AA68A047041E61
:107A0000C6D1AB78029A5B08013BDB00D318390082
:107A100030005B689847041E0BD1AB78042BB6D0BE
:107A2000039A310010782200009700F06DFB0400EB
:107A3000AEE76A78002AABD1AA7805A93B8808711D
:107A400030000A704B80FEF747FBA0E71046FF1F8F
:107A5000E8C000111D4B37B5050098420BD0002936
:107A60000AD1FFF777FF002805D11948FFF772FF09
:107A7000002800D0058037BD01291AD1FFF76AFF21
:107A8000041EF8D001235B420380A378FF2BF2D0C1
:107A9000FE2B07D00023E0781422009329001E3328
:107AA00000F032FBA01C00F054FB01235B4263801A
:107AB000E1E70229DFD1013901F0BEF80028DAD16F
:107AC0002800FFF747FF041EDFD1D4E7FEFF0000C8
:107AD000FFFF0000022210B5074B52421A800748F0
:107AE00001325A809A80DA8000F07EFA044801F070
:107AF00025F8002010BDC046C067FF1F797900112E
:107B0000557A00110388F7B50400002B02D1022535
:107B10002800FEBD42680221137825485268FEF70E
:107B2000A5FD00282ED0234F01253A88002AEFD04A
:107B3000802321885B0201259B1A9942E8DC0C20F6
:107B400003F0D6FF061E31D03B8822889C460023D6
:107B50001800019561469DB2491989B2AA421BD805
:107B6000002801D062443A8000233000082208C077
:107B7000210004F055F9104A1368002B13D1002599
:107B80001660C5E76268022113780C485268FEF758
:107B90006DFD0028C7D1BAE760681D014019418119
:107BA00001330198D6E71A001B68E6E71325AFE713
:107BB00056C100110E46FF1FBC67FF1F54C10011C4
:107BC000014B18707047C0461046FF1F14230A006F
:107BD00010B51A40194204D00122102101F048F8D2
:107BE00010BD4B06F9D4012088434000F8E710B5DA
:107BF00014008B0604D50122102101F039F810BDC4
:107C000008230A001A40194202D14BB2002B0FDAA6
:107C1000102101F02DF8002808D02300F9331B783B
:107C2000002BECD0F8342378012BE8D10020E6E7D4
:107C300003208907FAD4E2E7F0B51F00184B85B09E
:107C40001C68019002910392002C27D1200005B0FE
:107C5000F0BDA5683301ED186B89019A934211D3E9
:107C6000029A93420ED8002F04D10A9B002B10D108
:107C70002C00EBE73B002978039A6868FEF7F6FCD6
:107C80000028F2D10136B6B2A388B342E1D8246805
:107C9000DAE7A3680A9A5B891380E9E70026F3E72D
:107CA000BC67FF1F37B50C000A8849880123914241
:107CB00017D3002A15D0651D23792A0002210A480E
:107CC000FEF7D4FC102300280BD02379618820888C
:107CD00000242A000094FFF7AFFF0A23A04200D03F
:107CE000230018003EBDC04656C1001113B50A005E
:107CF00008884988012388420BD8002809D000242D
:107D0000137905320094FFF797FF0A23A04200D0B1
:107D10002300180016BD13B50A00088849880123FE
:107D200088420BD8002809D000241379053200942A
:107D3000FFF782FF0A23A04200D02300180016BDDF
:107D4000F0B58BB003904A8808880E000123824268
:107D500055D3002853D00023012704AC2370002200
:107D6000718813000092FFF767FF051E3ED0207850
:107D7000002835D12B78022B18D167706A898300CF
:107D80000130E31880005A8069680222201804F04C
:107D900047F823780133DBB22370042B19D93B0059
:107DA0006889013080B2002BD9D01FE002236370B4
:107DB000122358436A89231804305A8069681022B4
:107DC000201804F02DF823780133DBB22370002B48
:107DD000E5D10C4A6B899B185A425341DBB2DFE76D
:107DE0006378012BE4D12B78022BC7D022780A23A9
:107DF000002A04D021000398FEF798F90023180008
:107E00000BB0F0BD0100FFFF0F4BF0B50400186888
:107E1000002816D083685D89A54207D88288AE18ED
:107E2000B44203DA12019A18934201D10068EFE7D5
:107E30001E005F891036A74204D1002900D00D80B2
:107E40001800F0BD3300EFE7BC67FF1F70B50500F9
:107E50000C0008880021FFF7D7FF03000120002B4A
:107E600004D022002800197AFFF7C1FE70BDF7B5D3
:107E70000C00002501902300F6331B78AB4201D89B
:107E800000200AE06B00E65A00213000E718FFF7F7
:107E9000BBFF002802D126800130FEBD017A019887
:107EA000FFF794FE002802D03B882380F5E70135D8
:107EB000EDB2E0E710B5040008880021FFF7A4FF49
:107EC00003000120002B03D02000197AFFF77EFE6B
:107ED00010BD0000054B1B68002B01D1180004E009
:107EE0009A6852898242F6D198887047BC67FF1F12
:107EF000F0B50E27002687B0039302ABFF183E8033
:107F000005001F4B40891400984207D02B780130A0
:107F100000976A6880B2FFF78FFE060002212B7877
:107F200018486A68FEF7A2FB00280FD06C89200071
:107F3000FFF7D0FF002802D0013C0419A4B2039B34
:107F4000002B00D01C80300007B0F0BD02212B7840
:107F50000D486A68FEF78AFB0028E7D102212B78DA
:107F60000A486A68FEF782FB002807D0002EDED0A0
:107F70003B88A342DBD17489013CDFE76C89DEE7F3
:107F8000FFFF000056C1001154C1001152C1001181
:107F900010B50C00FFF7DEFC03000220002B0AD016
:107FA000002C00D023609B781720FE2B03D00138D3
:107FB000FF2B00D1002010BD73B50D0001A90400F6
:107FC0001600FFF7E5FF172805D0002E04D1290081
:107FD0002000FEF727F976BD01221021200000F0D5
:107FE00047FE0028F3D0F6E7014B18607047C04603
:107FF000CC67FF1F37B56B469D1D010004000222B0
:10800000280003F0C5FD2B88B02B0ED12379122B4D
:1080100009D12300FF339B78012B06D10121608811
:1080200000F0E0F801E01B2BF8D037BD10B5054B90
:108030000421187000F098F8FFF74CFDFEF770FB74
:1080400010BDC046D067FF1F0020F0B50BB20F0077
:1080500087B0834234DA274B187803F0E9FD051E18
:108060002BD00378A02B25D103AE3100FEF7E4F826
:10807000041E0BD1B378DB0724D51F4B06341B68D5
:10808000002B03D03100688898470400A8680028B6
:1080900001D003F0CDFE002C08D1184A039B1340F9
:1080A000174A934206D0B3781B2B03D0012168886E
:1080B00000F098F8280003F0ABFC80200002784024
:1080C00007B0F0BD0F4B1B68002B10D03100688843
:1080D0009847041EDAD07378002BD7D1B27801A963
:1080E0000A704B800C716888FDF7F6FFCEE7062416
:1080F000F1E7C046D067FF1FC867FF1F00FFFF0002
:1081000000011200CC67FF1FF7B5019082204000EC
:108110000D0017001E0003F073FC04001320002C58
:1081200012D0B02320002370089BFC22677065806A
:1081300026710830002B08D0190003F071FE2100D1
:10814000019803F02DFD0020FEBD089903F070FC9E
:10815000F5E710B5041E06D00078FD2803D803F01B
:10816000BFFCFF23237010BD0A1F93B210B504009B
:108170000220032B05D882400020024BD1529B18CD
:108180009C7010BDF067FF1F0B8870B5043B0400A6
:108190000D000220032B0BD80121200000F04CFD24
:1081A00003001420002B03D02900200000F0DEFB88
:1081B00070BD000007B51300034A00920A000121B8
:1081C00000F02CFC0EBDC046F183001107B50192F2
:1081D00003220092024B0A00122100F049FC0EBD5E
:1081E0006F84001107B56B4601AA11800449D8803D
:1081F00008780633012802D1190003F031FD07BDCC
:10820000D167FF1F0C4B10B518700023FF210B4ADC
:108210001380138193819380094A538013705172A4
:1082200093819372D174D3821375517703F0D0FD8B
:1082300000F0FCF910BDC0460068FF1FF067FF1F8B
:10824000D267FF1FF0B58DB06B46002003910C2262
:108250009B5E834200DBB0E05D4B187803F0E8FCE6
:10826000051E00D1A4E00378902B00D09DE006AF5E
:1082700001004688380000F013FA796804000029EC
:1082800000D19CE03B88052B6ED13B89032B1CD988
:1082900005AC200000F0A2F86288172A61D839895D
:1082A000131D994231D17968237804310291D9079D
:1082B00038D5607800F08EF9071E06D000230371D0
:1082C0002378012B08D0132B23D0A868002800D1D5
:1082D00078E003F0ADFD75E06288029909A800F02E
:1082E000A6F80290380000F08BF909AA2378387AB2
:1082F0000192002231000092029A00F012F9380037
:1083000000F064F9029B002BDFD0300000F080F910
:10831000DBE70378032BD8D16288029909A800F023
:10832000D6F8DEE7122B13D1029909A800F0B5F8B0
:10833000021EEAD127498B88002BC6D0887909A96B
:108340002378019161780091310000F0EAF8BCE7F0
:10835000002302AA93833000617809AAFFF72AFF5D
:10836000B3E71D4B0993F6E7042B02D09A1F012AAD
:10837000ABD8184A043B9B00995A0029A5D0D218C3
:10838000907831003A0000F0AEF800289DD13B888B
:10839000042B03D001213000FFF724FF012C04D16E
:1083A000A868002801D003F043FD280003F030FB4B
:1083B0008020039B0002434018000DB0F0BD01284F
:1083C00000D182E701213000FFF70CFFEDE7C04646
:1083D0000068FF1FF067FF1F010017000B78037094
:1083E0004B784370CB788A781B02134343807047E5
:1083F0000A88030002700A88120A42700A88012A59
:1084000006D14A8882704A88120AC27004207047D6
:1084100002208242FBD14A8804309A704A88120AAC
:10842000DA708A881A718A88120A5A71EFE710B5D1
:108430000400012082420CD94B780A781B021343B6
:108440002380834206D1CB788A781B021343638052
:10845000002010BD022BFBD1CB788A781B0213437E
:1084600063804B790A791B021343A380F0E70B88E2
:1084700003700B881B0A43704B8883704B881B0A60
:10848000C3708B8803718B881B0A4371CB888371FF
:10849000CB881B0AC3710820704703000120082AFB
:1084A00014D14A780878120202431A80CA78887870
:1084B000120202435A804A790879120202439A80D2
:1084C000CA798879120202430020DA80704710B519
:1084D00004000120022A05D100204B780A781B02F3
:1084E0001343238010BDF8B5060010200F001500BF
:1084F00003F086FA04000120002C0ED0A0230C22E9
:10850000290023806780201D002D07D003F088FC00
:108510002100300003F044FB0020F8BD03F088FA8E
:10852000F6E7F7B51E00009008AB142017001D7881
:10853000019103F065FA041E12D0A2230370019B7F
:1085400047704380099B057146710C220830002B4F
:1085500007D0190003F064FC2100009803F020FB11
:10856000F7BD099903F064FAF6E737B5041E0FD09A
:108570004388002B0CD00025C1881323007A1722D2
:1085800001950095FFF7CDFFFF236580637225708D
:1085900037BD000010B50C4904004A88002A09D0F4
:1085A0008B89002B05D00020CB8A0222834201D088
:1085B00010BD012213000A20434300204032C8545A
:1085C000C81842800472F3E7D267FF1F002343807C
:1085D00003707047094B00211A0010B55C88002C0D
:1085E00006D01C79844203D10A234B43D01810BD16
:1085F00001310A330329F1D10020F8E7D267FF1FC8
:1086000010B50400407A03F06BFAFF23637210BDCB
:108610007047043010B580B203F03AFC002803D054
:108620000421494203F034FB10BD000070B5002561
:10863000104CA0682580A581A580A84202D003F037
:10864000F7FBA56000250C4C0C4B606D1D802300D2
:1086500058331D70A84202D003F0EAFB656500257F
:108660006068002801D003F0E3FB013508340A2DCF
:10867000F6D170BD9868FF1F3C68FF1F8C68FF1F14
:1086800070B5041E09D1054D2880A881A880A8686E
:10869000002802D003F0CCFBAC6070BD9868FF1FCF
:1086A000F0B54B8885B00193002343600A7905003B
:1086B0000F00022A00D07BE0CA88032A17D98B68F2
:1086C0005E7819783602DC78D8790E4399781B7A6F
:1086D00024021B020C43034353495BBA0B80331D36
:1086E00093421ED1042C04D0631F022B0ED901200B
:1086F00015E0019A4D4B1201D35A002B06D0019878
:10870000FFF7BEFF4A4A1369013313610421B868B9
:108710002E812C80494203F0BBFA6860002005B02E
:10872000F0BD434D042C06D0631F022B0FD9EB681C
:108730000133EB60DBE7019A3C4B1201D35A002B6B
:1087400005D00198FFF79CFF2B6901332B61374B54
:1087500030000293019B029A1B01019300230199AF
:108760008C468B52130063449C8003939E81FFF7D9
:1087700050FF039B041E986016D00421B86849423C
:1087800003F086FAFA880100043A200003F048FB5F
:108790000199029AFB888A5A043B9B18029A8B52D1
:1087A0002B6801332B60A2E7AB690133AB619EE715
:1087B0001E4B0293019B1E01029BF35A002B2DD0EE
:1087C00002998C19A068002828D0012A26D1FA889D
:1087D0009B189BB27352A189994217D39B1AC01858
:1087E000B96803F01DFB029BA289F35A934200D0A3
:1087F0007DE700222B81A3882B80A3686B60029BFE
:10880000F2520B4A53680133536070E7084A936889
:10881000013393600198FFF733FF68E7044A536917
:1088200001335361F6E7C0460268FF1F9868FF1FD7
:108830000868FF1F70B5051E15D10B4C0B4B188037
:10884000230058331870606D002802D003F0F0FA4E
:108850006565250050356068002801D003F0E8FA0E
:108860000834AC42F7D170BD3C68FF1F8C68FF1F15
:10887000F0B51700A12285B0920001934243394B15
:1088800006001B680C009B18D933FF331D78FDF7D9
:1088900041FF0430854204DD3000FDF73BFF04302A
:1088A000C5B2BD4207D33A0000213000019B03F05E
:1088B00027FA05B0F0BD2900380002F0E9FF2300D7
:1088C000C6B250331E700393019B290063653800C4
:1088D00003F04EFACBB20293002B02D0039B013679
:1088E0001E7000262300503303931B78B34204D834
:1088F000606D002831D10020DBE7029A2800002AB1
:1089000004D0013B1000B34200D02800F700E71963
:10891000387003F015F8786000280ED03A78019985
:1089200003F07EFA019A3B780136D3180E4A019380
:10893000D369F6B20133D361D4E7039B1870606545
:10894000A74205D1084A1320D36A0133D362B0E7A6
:10895000606803F06DFA0834F2E703F069FA002367
:108960006365C8E73409FF1F0868FF1FF7B50D00EE
:1089700007000421686803F08BF92B890400037059
:108980002B891B0A43702B8883702B881B0AC370AA
:108990002E8902250436F6B2FB2E15D81B4B9F42BA
:1089A00014D10C2003F02CF81135011E0CD09023AB
:1089B00003708E3B0371043B4380154B8460C6807B
:1089C000187803F0EDF800252800FEBD5C237B43FA
:1089D000104AD3180093583301931B78002B0FD102
:1089E0000300320038000099FFF742FF019B0500A9
:1089F0001B78002BE8D13800009902F031FFE3E743
:108A0000054A0725536A01335362DDE7FEFF000084
:108A10000068FF1F3C68FF1F0868FF1FF0B587B0A4
:108A2000009017200F0016000193FFF7F2FD1325A9
:108A3000041E19D00C98031E02D00199201D9847DE
:108A4000030AE370052302AAA07004309081277006
:108A50000098667003A993800494FFF787FF051EB2
:108A600002D0200003F0E4F9280007B0F0BD0000B8
:108A7000F0B587B01F000CAB1B7803910593012163
:108A80000DAB06001C78049200F0D6F814250028DF
:108A900021D02000FFF77EFD0135041E1BD01149B7
:108AA000059B0A7803700132D2B2131EC68001D131
:108AB00001231A000B7022713000049B0399009768
:108AC000FFF7ACFF051E09D1230021000648074A25
:108AD000093303F08DF8280007B0F0BD0023638050
:108AE0002370F8E70468FF1F6B85001130750000E4
:108AF000F8B505000E00064C064F2368002B02D087
:108B00003100280098470434BC42F6D1F8BDC04675
:108B1000A868FF1FBC68FF1F0123064A5B42538001
:108B2000002313715362044A136053609360D3604F
:108B300013617047BC68FF1FA868FF1F0200002375
:108B400010B506499C000859002801D1625010BD9B
:108B50000133052BF6D11320F9E7C046A868FF1FA3
:108B6000034A5388181A4342584140421040704704
:108B7000BC68FF1FF0B585B002930AAB1F780CAB41
:108B80001B88009008000E0001920393FFF7E8FF96
:108B900005001120002D1BD10E48FFF7E1FF040056
:108BA0001520002C14D006220B99A771E01D03F0AC
:108BB00037F9019B30002371029B29006371009BF0
:108BC00066802370039B6562E381FFF791FF2800B5
:108BD00005B0F0BDFFFF000010B5FFF7C1FF0400B6
:108BE0000220002C12D060880121FFF781FF606A0B
:108BF000002801D002F06CFE28220021200002F0A3
:108C000017FF012300205B426380207110BD00002C
:108C100030B5074A074C5588010013780020A5425B
:108C200004D05B1A59424B415842104030BDC046F7
:108C3000BC68FF1FFFFF0000084A10B501230C00AD
:108C4000904208D0FFF78CFF031E04D00379234025
:108C50005A1E9341DBB2180010BDC046FEFF000053
:108C6000024B1879431E9841C0B27047BC68FF1F81
:108C700070B504000D001600FFF772FF002804D144
:108C80000D4B9C4200D0143070BD416A0379052021
:108C9000002907D012221A40102A02D10520002EE6
:108CA000F2D10F20DB06EFD5897E0C20A942894145
:108CB000494249420840E7E7FEFF0000030010B5C3
:108CC000002800D110BD0348034A41889142F9D0E1
:108CD0009847F7E7BC68FF1FFFFF0000002330B58F
:108CE000C45CCD5C6C40D4540133102BF8D130BD42
:108CF0000F23002210B5C45C64002243CA54C25C36
:108D0000D209013BF7D210BD0200010010B520329C
:108D1000103102F0CDFF10BDF0B58BB003901020E4
:108D200005931700049102F0E3FE0090102002F07A
:108D3000DFFE009B13240190002B05D000280CD1EE
:108D40001324009802F0C4FD019B002B02D01800F0
:108D500002F0BEFD20000BB0F0BD102002F0C8FEF6
:108D60000600102002F0C4FE13240500002E00D1DE
:108D7000AEE0002819D01022002102F059FE320086
:108D80002900039802F094FF041E0ED133787F2B44
:108D900051D830000099FFF7ABFF009B1B787F2B69
:108DA00053D801990098FFF7A3FF300002F090FD1F
:108DB000002D02D0280002F08BFD002CC1D1102024
:108DC00002F096FE0600102002F092FE0290002EA5
:108DD0007CD0002878D03A000F32230001251211F0
:108DE00005D00F333B4015B25A4253411BB26A1EA5
:108DF0001201002B33D0049BD2B298180099029A2A
:108E0000FFF76CFF013D10220021300002F010FE40
:108E1000ADB2049F2D017D19AF4242D0002C33D05A
:108E2000300002F055FD029B002B00D189E71800AD
:108E300002F04EFD85E729003000FFF759FF2800BA
:108E40002549009AFFF74AFFA7E729000098FFF796
:108E50004FFF28002049019AFFF740FFA5E70F21A7
:108E60000F4004998A18D9B28F4208D9D15C06A85C
:108E700019540133102BF6D1029A0199C0E7791ADF
:108E800048424141C901F2E73900300006AAFFF724
:108E900025FF3200039806A902F00AFF10370400EC
:108EA000BAE7002CBCD13000029906AAFFF716FFE2
:108EB000320006A9039802F0FBFE082204003100EC
:108EC000059802F0ADFFABE71324A9E71324AAE746
:108ED000002800D06EE733E75CC10011F0B58BB01D
:108EE0000F0016000225009000283FD0002A3DD038
:108EF0000B1DDBB21800029302F0FAFD1135041EBF
:108F000034D0FDF747FD05003A000099201D02F01E
:108F10004FFEEBB20393E3702B0CDBB22F0A0093EE
:108F20006370FFB22B0E2370A7700193FDF72CFD29
:108F30001022010006A802F03BFE2100029A04ABB9
:108F400006A8FFF7E9FE051E0DD1039B082233702A
:108F5000009B04A9B370019B7770F370301D02F081
:108F600027FEFDF71DFD200002F0B2FC28000BB02B
:108F7000F0BDF0B58FB00D00149E039004920593E0
:108F8000002A03D1022420000FB0F0BD002EF9D03A
:108F90000398FFF7E5FD1424071EF4D072783378A8
:108FA00012021A43B3781B041343F27812061A43D1
:108FB000036A0192934201D30133E3D1002D03D020
:108FC0003B7901249B07DED50822002106A802F088
:108FD0002FFD059B13240433DBB21800029302F02B
:108FE00087FD051ECFD0059A0499043002F0E0FDFC
:108FF00004223100280002F0DBFD3900102210317C
:109000000AA802F0D5FD2900029A06AB0AA8FFF7CC
:1090100083FE041E0FD1082206A908A802F0C8FD8D
:109020000822311D08A802F013FC012807D101997C
:109030000398FDF7C9FC280002F04AFCA3E70124CD
:10904000F9E7000070B51C4C05002368181E10D00D
:10905000002D14D11A78002A0CD1981C083202F085
:10906000DFFE02F01DFC0135002808D123681D70C9
:10907000012070BD0A331800082202F0D1FE2368D7
:10908000002BF5D0122002F0BBFC061E0DD0C12330
:1090900021680370457002311022023002F0C0FED8
:1090A00023683100587802F07BFD206802F010FC44
:1090B00000232360DCE7C046E468FF1FF8B5040026
:1090C0002020FDF755FB0D4EA700BB590500002BD6
:1090D0000DD000280BD0D878FF2809D108492A00E4
:1090E0000C55F35907480333611802F081FDF8BDB0
:1090F000290002F075FE0028F0D1F8E70069FF1F93
:10910000E868FF1F15A3001170B5064D8400635970
:10911000002B05D0D87802F0E3FCFF226359DA7007
:1091200070BDC0460069FF1F70B506008CB00C0012
:10913000150000213022684602F07AFC310010222E
:10914000684602F035FD1D2021000322684402F02C
:109150002FFD6846FFF7D8FD2D21040003222800CB
:10916000694402F025FD20000CB070BDF0B5070089
:10917000160097B001931CAB1D7830221EAB0091F6
:109180000AA800211C7802F053FC102239000AA81A
:1091900002F00EFD1022002102A802F049FC072275
:1091A000310002A802F004FD072202AB9818631EEA
:1091B0009C41019902F0FCFC02AB9C732B005A1EEF
:1091C000934102AAD3730021102206A802F030FCBA
:1091D00006221D9907A802F0EBFC1A2002ABC0186A
:1091E00006221F9902F0E4FC102200990EA802F05A
:1091F000DFFC102202AB0EA908781C78013A60400F
:10920000D2B2087001330131002AF5D10AA8FFF764
:109210007BFD102212A904000EA802F001FE10220C
:1092200006AB0EA908781D78013A6840D2B20870E2
:1092300001330131002AF5D10AA8FFF765FD044387
:1092400010222098E4B212A902F0B2FC200017B05C
:10925000F0BD70B50E0014008CB0010010226846FD
:109260001D0002F0A5FC3100082204A802F0A0FCB9
:109270002100082206A802F09BFC6846FFF744FD87
:1092800004001022280008A902F092FC20000CB073
:1092900070BDF8B506000D0000243719AC4200D3AC
:1092A000F8BD02F0D5FD030A3B70631CDBB2013749
:1092B0009D4203D90234F054E4B2EEE71C00EDE71E
:1092C00073B506000C000225002819D0002917D01C
:1092D000032101A8FFF7DDFF6B469A793F231A406F
:1092E000013313436A463000937101A92200FFF74E
:1092F0001BFF051E04D10322E01C01A902F090FD12
:10930000280076BD03785807DA08C00FD200800025
:109310009B0710439B0F1843C0B2704707230B40B5
:10932000C908C9000B4303707047000070B5040002
:10933000FFF7EAFE134DA4006359002B21D0186AF1
:10934000002801D002F0C4FA2B59986E002801D0F1
:1093500002F0BEFA2B59D86E002801D002F0B8FAFC
:109360002B59186F002801D002F0B2FA2B59586F10
:10937000002801D002F0ACFA285902F0A9FA002323
:109380002B5170BD0069FF1F0E4B8000C35870B594
:109390000C00002B0FD09D68002D0CD02B78201DC9
:1093A0000B706B784B70A97CFFF7B8FF2B7E237294
:1093B0006B69E36070BD10220021200002F038FBD1
:1093C000F8E7C0460069FF1F014B18607047C046B0
:1093D000FC68FF1F074A03008000825810B5002A6E
:1093E00006D0D088984203D1012901D1FFF79EFF12
:1093F00010BDC0460069FF1FF0B5264E95B087002E
:109400000B93BB590500099112200A92002B31D011
:10941000D888FFF7A5FB04001420002C2AD02800D0
:1094200010A9FFF7B1FFBB591E781D6A002E23D08B
:109430000895FDF7EFFA07000020FDF7F1FA079015
:10944000A379E61D069310AD0CA9089800F0E2FA86
:109450000EA9280000F0D7FA0B9B0A990493069BEB
:1094600009980293079B0396019300970EAB0CAAF1
:10947000FFF77CFE15B0F0BDFDF7CCFA069030008A
:10948000FDF7CEFAE31DA779079310AB060008930A
:10949000DAE7C0460069FF1F30B50C4C85002A5939
:1094A000030085B00120002A0ED018006946FFF79E
:1094B0006BFF2B591A78D888054B002A00D1054B31
:1094C0006A46072100F0D9FB05B030BD0069FF1FD7
:1094D000079A0011159A001130B5094C85002959D9
:1094E00085B010226846253102F09AFC2A591121D4
:1094F000044BD0886A4600F0C0FB05B030BDC046C2
:109500000069FF1FB19A001130B5094C8500295937
:1095100085B010226846353102F082FC2A591121AB
:10952000044BD0886A4600F0A8FB05B030BDC046A9
:109530000069FF1FEF9A0011F7B54D4F860010200C
:10954000F4590D0002F0D4FAF3592062186A13227C
:1095500000286CD0033A29009C6802F061FCF359A2
:109560001A780192002A58D11E6A227D317B9446D6
:1095700051400122019F114201D167461740217DD0
:10958000914339432175377B4F40BC4660460027E5
:10959000800701D44F081740012102208F40227D0F
:1095A00082433A432275377B5740BC4660460027CA
:1095B000400701D497080F400420227DBF0082435A
:1095C0003A432275627D002794466046727B424092
:1095D0000A4201D167460F400121627D8A433A4326
:1095E0006275777B5740BC4660460027800701D4F0
:1095F00057080F400220627D7F0082431743677542
:10960000767B00227E40760701D4BA080A40042601
:10961000617D9200B1430A4362756A78002A08D0DE
:109620006278002A05D005220533DA77002210007F
:10963000FEBD04222979114205D1A17C114202D13B
:109640000533033AF1E7019A21782C78002A02D1F8
:109650000A002100140018220429E8D8042CE6D8B6
:1096600005206043034A05331218525CDDE7C0460B
:109670000069FF1F6CC1001110B50A001121024BD7
:1096800000F0FBFA10BDC0464B9B00110B0030B53B
:1096900087B001AD2B806B4604001100981D082295
:1096A00002F0BEFB2A000B212000024B00F0E5FA7D
:1096B00007B030BD739B001110B50A001121024B99
:1096C00000F0DBFA10BDC046C79B001113B50B00BC
:1096D00011006A4613706B4604000622581C02F003
:1096E0009FFB6A4608212000014B00F0C6FA13BD1B
:1096F000E79B001110B50A001121024B00F0BDFAE2
:1097000010BDC046379C00117FB505000B4BAA0069
:10971000D4580800002C0FD0666F237FE288217890
:109720000396266F0296E66E0196A46E0094FDF7EE
:1097300009FC2800FFF7FAFD7FBDC0460069FF1F46
:1097400010B51721FFF7E0FF10BD000070B50A004B
:109750000D00064B0221040000F08FFA0600297864
:109760002000FFF7D1FF300070BDC046179B0011ED
:1097700070B586B000236A461370836804001D78B4
:10978000681E0A2859D801A902F092F80606333754
:109790003B3F43474B4F5300180000F042F906236C
:1097A00012284BD000281BD16088FFF7D9F9082375
:1097B000002813D04279002A47D1264B1A78072374
:1097C00012070BD5244B1A680723002A06D0166807
:1097D000002E03D0290001AAB04703006A46137087
:1097E0006B461B786088002B2AD1FFF767FC06B018
:1097F00070BD180000F06CF9D4E7180000F087F98C
:10980000D0E7180000F093F9CCE7180000F0ADF9AC
:10981000C8E7180000F0C3F9C4E7180000F0F6F933
:10982000C0E7180000F0F6F9BCE7180000F013FAE2
:10983000B8E7180000F013FAB4E707236A4613707C
:1098400069466088FFF782FFD1E70523012AC5D169
:10985000024BB8E78D67FF1FF868FF1FFC68FF1F0A
:10986000F8B52C4F8600F35904000D00002B40D0B2
:10987000DA8882423DD15A78062A33D11A78002AF2
:109880002ED0012099681A6A097D014206D0157B05
:10989000054203D007225A700120F8BD0220014280
:1098A00004D0157B054201D00922F4E704200142CF
:1098B00004D0127B024201D00B22ECE7164B1B684E
:1098C000002BE9D05B68002BE6D020009847BB59FD
:1098D00000215B78122BDFD12000FFF715FFDBE7BB
:1098E0000E4BECE7112A04D1002900D032252900C3
:1098F000F2E7002D08D12000FFF732F9002803D04D
:10990000102302791343037121002800FDF798FA10
:10991000C2E7C0460069FF1FF868FF1FFC68FF1F11
:1099200070B50E4E8500AB590400002B13D01B7888
:10993000002B11D10A4B1B68002B04D05B68002B55
:1099400001D02000984773595B78122B03D1002176
:109950002000FFF7D9FE70BD024BECE70069FF1F46
:10996000FC68FF1FF868FF1F094B8000C3581020D8
:10997000002B0CD01A6A002A09D09B68002B06D055
:10998000127A1B7E101C9A4200D9181CC0B2704774
:109990000069FF1F70B503000D0014000220002AAB
:1099A00030D000292ED013700B78081D53704B78DF
:1099B0009370FFF7A7FCE070012002212B7A23713E
:1099C0006B7B034063716A7B0A401343042263711B
:1099D0006E7B1640334363716E7BF608F6003343AB
:1099E00063712B7B0340A371287B014000200B4354
:1099F000A371297B0A401343A3712A7BD208D200AA
:109A00001343A37170BD10B50A0001000120FFF7D8
:109A1000C1FF10BD10B50A0001000220FFF7BAFF18
:109A200010BD70B506000C000220002E30D00029B9
:109A30002ED07378201D0B70B3784B70F178FFF740
:109A40006DFC01223579257271794B1008001340A5
:109A5000934010400343881010408000C90803431E
:109A6000C9000B436373B1794B1008001340934056
:109A700010400343881002409200C9081343C900F4
:109A80000B4321202373FCF773FE854201D2122081
:109A900070BD2220257AFCF76BFE8542F7D823782B
:109AA0001820042BF4D86378012BF1D80020EFE7BD
:109AB000030010B50220002909D0002B07D0032293
:109AC000481C0A7019000D3202F0AAF9002010BDDE
:109AD00003000222080010B5002B06D0002904D094
:109AE0000E32591C02F09CF90022100010BD030038
:109AF00010B50220002909D0002B07D00422481CF1
:109B00000A7019000C3202F08BF9002010BD10B55C
:109B1000FFF7DEFF10BD03000220002906D0002B56
:109B200004D0052200200A701B784B707047030098
:109B30000220002B08D0002906D05B7800200B7093
:109B4000013B082B00D918307047030010B50220E4
:109B5000002909D0002B07D00622481C0A701900E2
:109B60000A3202F05DF9002010BD10B5FFF7B0FF1A
:109B700010BD02000B00022010B500290ED0002AF3
:109B80000CD007211970118859701188090A997031
:109B900011180822D81C02F043F9002010BD030060
:109BA0000A00022010B5002B0CD000290AD09978A9
:109BB0005878090201431180901CD91C082202F038
:109BC0002FF9002010BD030010B50220002909D094
:109BD000002B07D00822481C0A701900921802F0C6
:109BE0001FF9002010BD02000B00022010B5002953
:109BF0000BD0002A09D00921197011781818597052
:109C0000511C062202F00CF9002010BD10B5FFF720
:109C10005FFF10BD02000B00022010B5002A09D022
:109C2000002907D05178197011180622581C02F02B
:109C3000F7F8002010BD030010B50220002909D05C
:109C4000002B07D00A22481C0A701900063202F0C5
:109C5000E7F8002010BD10B5FFF73AFF10BD020075
:109C60000B00022010B5002A06D0002904D01800ED
:109C70005178FFF753FB002010BDF0B585B01700F9
:109C80001E006A4606230500080091819380FEF7B6
:109C9000C0FC1324011E02900CD03800B047041EF3
:109CA00005D1280001A9FEF76FFA041E02D0029820
:109CB00002F0BEF82800FFF701FA200005B0F0BD61
:109CC000F0B504008BB0019115000021102202A80C
:109CD00001F0AEFE334EA700B85900283CD0C3882F
:109CE000A34239D10378002B36D14278062A18D105
:109CF00002000100553235310C3006ABFFF7A9FAEE
:109D0000002829D12000FFF72FFE020006A902A893
:109D100002F086F8200002A901F0BAFE01200BB083
:109D2000F0BD816E002917D00B8A112A28D19D42DF
:109D30000ED101981231093A01F08AFD012807D1AC
:109D4000BB5920009D6EFFF70FFE29000200DEE7E1
:109D500032212000FFF7D8FC2000FEF701FF061E8D
:109D60001BD0416A002918D00B8AAB4215D10822BA
:109D70000198123101F06CFD01280ED1716A0AE0E0
:109D80009D42E9D108220198123101F061FD0128BC
:109D9000E2D1BB59996E8A7EB9E7200001F038FF05
:109DA000BCE7C0460069FF1FF0B56B4D87007E59C8
:109DB00085B0337802900393002B00D087E0B3681E
:109DC000346A01937078062817D101221B7D134253
:109DD00002D0217B114218D10222134202D0217BF2
:109DE000114251D10422134203D0237B134200D0ED
:109DF0008BE0019B5A7DEB5991E007380428F8D895
:109E000001F056FD032E42678300B36E002B03D191
:109E10001C2001F06DFEB066EB599C6E002C1CD02E
:109E200010220021200001F003FE0298FFF79CFDA4
:109E300001002000FFF72DFA02F00AF8208220002E
:109E400008211230FFF725FA0298FFF78DFDA07662
:109E5000EB592100D888FFF70FFC0822EB591CE0D2
:109E6000B36E002B05D01A00198AF0881232FFF762
:109E70000DFC0222019B197DEB5911423DD0207B44
:109E800010423AD0073208E0F488FCF7DBFD01000D
:109E90002000FFF711FC0A22EB595A70029B9C002C
:109EA0002A595378073B042B11D8D088FEF758FE67
:109EB00000284ED0C3895A08D2182849029B02981C
:109EC000CB542B5941180433254801F091FE05B0BD
:109ED000F0BDFCF79FFD03000120834201D100206B
:109EE0000393EB59DE88FCF79BFD039902003000D9
:109EF000FFF7ECFB019AEB59117D042211420CD0C3
:109F0000217B114209D00B22C7E7F688FCF73CFD04
:109F100001003000FFF7EEFB6BE7019A527D012153
:109F20000A4204D0607B084201D00C22B5E702212E
:109F30000A4204D0607B084201D00E22ADE7042122
:109F40000A4204D0627B0A4201D01022A5E7122205
:109F5000A3E7FA225200B0E70069FF1F0469FF1F60
:109F60001FA3001110B5064B1A78042310001840E7
:109F70001A4200D00348FFF727FA002010BDC04660
:109F80008D67FF1F1446FF1F70B50400FFF7D4FA5A
:109F9000051E43D12000FFF77FFA234EA400A059ED
:109FA0008268937CDB0708D50321036A1B790B4089
:109FB000012B02D1017F0B430377431DD97F8B1EF9
:109FC000022B0DD8022900D00121C088FCF790FF98
:109FD000042133591A7F59700A431A77280070BD3B
:109FE00001290CD102231022437000210C3001F012
:109FF0001FFD305910213530FFF74BF9EEE70529E9
:10A00000ECD10223D118437010220C3001F008FF6C
:10A0100004233259117F0B431377EAE708251828E8
:10A02000DCD1053DDAE7C0460069FF1FF0B58BB013
:10A03000059143887E4F9E00F45915000493002C2F
:10A0400015D1012902D000200BB0F0BD101D5778AA
:10A050001678FFF757F9EB68320002932B7A0499D0
:10A06000019300903B002000FCF70CFFEBE7E38836
:10A07000049A934201D00820E6E72378012B00D10F
:10A08000D4E0059B581E092800D9CFE001F010FC50
:10A0900005CE0A29CC506C859AB229000498FFF7A6
:10A0A00073FFD1E7200029001022453001F0B8FEEF
:10A0B000B9594B78042B02D1013B4B70C3E70B001D
:10A0C0000A00253335320C310498FFF795F90498CE
:10A0D000FFF702FA0522431E9841BB59C0005A708F
:10A0E000B2E7200029001022553001F099FE049BB0
:10A0F0004F4C9D00295904980A0006AB55320C318B
:10A10000FFF77AF929591022453106A801F0A0FB82
:10A11000012808D10498FFF7F7F90590002804D129
:10A1200006222B595A7005988EE708230593FAE703
:10A1300063780C2B7AD1E36E002B03D11C2001F045
:10A14000D7FCE066BB59D86E00286FD010222900DA
:10A1500001F066FEBB590498DC6EFFF705FC0D228A
:10A16000A076BB595A706EE7E06E00285ED0637827
:10A170000D2B5BD12B8808220382A91C123001F021
:10A180004FFEBB599A68517D0222114226D0186AAF
:10A19000407B104222D00C32E4E763780E2B45D18D
:10A1A000236F002B03D1162001F0A2FC2067BB59BE
:10A1B000186F002803D01022290001F031FE0F2271
:10A1C000BB59CFE763780F2B30D1206F0622691C73
:10A1D000103001F025FEBB599A68517D04221142CE
:10A1E00003D0196A497B1142D5D100210498FFF7A9
:10A1F0008BFA28E7636F002B0DD0BB59586F0028EE
:10A20000F3D01022290001F00BFE0122BB5952426B
:10A210005B6F1A61E9E7142001F06AFCBB596067C3
:10A220005B6F002BE9D126E72978DFE707200BE7F2
:10A230000069FF1F10B5064C207001F001FC0621DB
:10A240002078FDF791FF0348FEF778FC10BDC0466B
:10A250001369FF1FD593001100200BB270B50D00DC
:10A26000834216DA264B187801F0E2FC041E0DD06A
:10A270000378922B0ED0A02B37D0224B1878FF28D2
:10A280003AD0210001F08CFC002835D1802000025A
:10A29000684070BD43780E2B0BD03E2BEDD18378F8
:10A2A000052B12D0082BE8D181798088FFF7D8FAE6
:10A2B00008E0154B82889A42DFD183681878591CD0
:10A2C000FEF7C0FE002817D1D7E7104B1B785B07BD
:10A2D00012D50F4B1B68002B0ED09B68002B0BD0A8
:10A2E000C289811D80889847ECE7FFF741FAA06892
:10A2F000002801D001F09CFD200001F089FBC5E79A
:10A300001369FF1F0D46FF1F182000008D67FF1FF8
:10A31000FC68FF1F10B50078FFF712FA10BD10B5EA
:10A320000078FFF7FDFA10BD0C234343084A10B52F
:10A330009B185A68002A03D0012901D1904710BD0B
:10A340009B68002BFBD00029F9D19847F7E7C0465E
:10A350003069FF1F01238340094A10B5946B1C43E9
:10A360009463506B98435063D46B20009843012949
:10A3700001D120001843D063116B0B43136310BD50
:10A3800000800040F0B500240127154B85B0DA6B42
:10A39000144E03921A6C0192DA64019BE3403B4233
:10A3A00017D0039DE5403D400295E5B20299280093
:10A3B000FFF7BAFF316A736A002908D03900002B11
:10A3C00001D0029979402800FFF7C4FF01E0002B7B
:10A3D000F9D101340C36172CDFD105B0F0BDC046E1
:10A3E000008000401469FF1F064B01215A68C240DB
:10A3F0000A4204D01B68C3401800084070471B6D18
:10A40000F9E7C046008000400122064B8240002947
:10A4100003D0D9680A43DA607047D9689143D9609C
:10A42000FAE7C0460038004030B5032444430F4BE0
:10A43000E25C1B199C785D7801232D1B0135AB4034
:10A44000013BA340A140DB430C00122807D8084978
:10A4500092005218116819402143116030BD054A1D
:10A4600011680B4023431360F8E7C046B3C10011E5
:10A4700008F0004014F00040C21F70B5D4B20623AB
:10A48000092C0BD80125084C9540002908D0002143
:10A49000FFF7CAFF23682B4323600023180070BD19
:10A4A0002368AB43F8E7C04600380040214BF0B5C5
:10A4B0001B185B78022B21D1032444431E4A1F4EF4
:10A4C000A35C12199478012215008540B76B013CFA
:10A4D000E4B23D43A240B563194C122815D89B0045
:10A4E00000290CD117495B1899680A439A60012327
:10A4F000205C154A834011680B431360F0BD11497D
:10A500005B18996891439960F1E70E4B00290DD1D2
:10A5100059690A435A61225C1328E8D00123203A82
:10A5200093400A49086803430B60E7E75969914380
:10A530005961F0E71469FF1FB3C1001100800040AA
:10A54000F8C1001100F00040A0F00040A4F000406D
:10A55000F8B500241B4E1C4D1C4B1B5D012B1FD15D
:10A56000194A9269E2401A420BD00122B256934036
:10A570002200143AD2B2022A09D815494A69134373
:10A580004B61013402360C35172CE5D1F8BD0022A1
:10A59000B2560F499200521891680B439360F0E74E
:10A5A000022BEED1E7B23800FFF71EFF012358401F
:10A5B000C1B23800FFF77AFF3800FFF715FF687760
:10A5C000DFE7C04685C100111469FF1F1569FF1F31
:10A5D00000F00040012202388240054B002903D0E0
:10A5E00059690A435A617047596991435961FAE7B9
:10A5F00000380040F8B50E0001210F008740114AD5
:10A600000400D368FD43BB43D360831E8B4201D853
:10A61000FFF7E0FF00212000FFF72EFF0A4A0B4B57
:10A620005168012E05D139431B1951605E7000201D
:10A63000F8BD2940516002221C1962709A691540C8
:10A640009D61F4E700380040008000401469FF1F5E
:10A65000012210B58240074B002906D019680A4331
:10A660001A600121FFF7C6FF10BD196891431960F8
:10A67000F7E7C046008000400C2370B50025434337
:10A680000A4A29009B181D70094B04001B185D70B5
:10A69000FFF7B0FF0123A340064928000A681A43C8
:10A6A0000A6005490A689A430A6070BD3069FF1F55
:10A6B0001469FF1F348000403080004070B50400F2
:10A6C0000E00FF2813D003250540FFF7D5FF084AE9
:10A6D000A3089B009B183F22ED00AA40AE401968DA
:10A6E00020009143314319600121FFF78DFE70BDB9
:10A6F00018380040F8B50C244443134B0500E41807
:10A700006368002B03D1A3681220002B1AD0022209
:10A7100001270E4B00215B195A7028002770FFF7A4
:10A7200069FF63681E1E08D0A3683E00002B04D09A
:10A730002800FFF759FE4640F6B228003100FFF727
:10A7400009FE0020F8BDC0463069FF1F1469FF1FD5
:10A75000F7B5C420FF222B4B8000195800249143E9
:10A760003F3A0A431A508022274F5202274E1A605E
:10A77000274B1D5D002D21D0A31E012B03D80121E5
:10A78000E0B2FFF727FF012D18D11F4B9B69E34073
:10A790002B4213D0E3B218000193FFF725FE01000E
:10A7A0000198FFF755FFE3B2143B022B1DD801219E
:10A7B0007156184A8D405369AB4353613B7F002B60
:10A7C0000DD0E5B22800FFF795FF2800FFF70CFE3B
:10A7D0007B7F0100834202D02800FFF7A5FD0134F2
:10A7E0000C370236172CC3D1F7BD01210023715657
:10A7F000F3568D40074A9B009B189A68AA439A60BB
:10A80000DCE7C04600E100E01469FF1F85C10011CC
:10A810001569FF1F00F0004070B50E001500040020
:10A82000FFF72AFF0C236343094A20009B189D6011
:10A830005E60FFF75FFFF021064B074A8900051EA7
:10A840005A5002D02000FFF717FF280070BDC04605
:10A850003069FF1F0000FF1F85A3001170B5134D65
:10A8600007202C78002C1FD19822210052002800AC
:10A8700001F04EF90123C420FF222B700C4B800005
:10A880001C635C630B4B1C605C600B4B1958914361
:10A890003F3A0A431A50802252021A600D20074A9A
:10A8A000074901F0A5F8200070BDC0461469FF1FDC
:10A8B00000800040A0F0004000E100E051A700113E
:10A8C00051A50011030010B50620072B09D8054A31
:10A8D000137001F0EDF8D7210020034B034A8900E3
:10A8E0005A5010BD3C46FF1F0000FF1F151BFF1FE5
:10A8F00070B51D0002240C2910D8094ACA40D2079D
:10A900000CD5FBF741FF041E08D1059A04992800D5
:10A91000FBF756FFFCF7C4FDFFF724FB200070BDDA
:10A920001210000030B50D7802232C009C43184211
:10A9300001D02B431C0008252300AB43284201D043
:10A940002B00234320241D00A543204201D01C439B
:10A9500025002A230D70184204D011781E3B0B43AA
:10A96000137030BD0028FCD10C2113788B43F7E71E
:10A97000F8B51D0006AB1B88140007AA0E000B20BB
:10A980001778002B27D10A78022A49D14A685078D3
:10A9900011780002244A08438018042840D800F0A7
:10A9A00087FF03121D1B2300F06800F0D1FF021C7B
:10A9B000C0B2B84200D93A1CD2B22000F1682A8055
:10A9C00001F02EFA06E00222F3681B882A80237029
:10A9D0001B0A63700020F8BD0622EEE701232B80DE
:10A9E000F3681B782370F5E7F368002B16D0082274
:10A9F0002A801A8822701A88120A62705A88A270F5
:10AA00005A88120AE2709A8822719A88120A627130
:10AA1000DA88A271DB881B0AE371DBE72B80D9E7B8
:10AA200001202B80D7E7C04600D6FFFFF7B5160000
:10AA30000A781D0008AB1F880C000123022A18D1D8
:10AA40004A685078117800022B4A0843801803287E
:10AA50000FD800F02DFF02254439E06800F078FFA0
:10AA6000C0B20723B84204D37B190193152B02DD32
:10AA70000D231800FEBDE0682A003100C01901F066
:10AA8000CFF96B4600209B88E268D0541B4B1B68B3
:10AA9000834203D01B68834200D098470023E8E735
:10AAA0000B23002FE5D1022DE2D1737832781B02FF
:10AAB0001343E2681380114B1B68002BEED01B6818
:10AAC000002BEBD00120E8E70B23002FD1D1062D7E
:10AAD000CED12A003100E06801F0A2F9DEE70B23B5
:10AAE000002FC6D1012DC3D132787533012AC0D8C9
:10AAF000E3681A70D2E7C04600D6FFFF206BFF1F45
:10AB000070B50C001500072837D800F0D1FE0414EA
:10AB100036361B36242E182015290BD8184E16222F
:10AB20000021300000F084FF22002900300001F0F5
:10AB300077F9002070BD18200229FBD11288114B33
:10AB40001A80F6E718200829F4D10A000E482900D7
:10AB500001F01EF8EDE718200129EBD10B4B10781E
:10AB60000B49DA69FFF7DEFEE3E718200129E1D19E
:10AB7000064B10780749DA6BF4E70220DAE7C046A3
:10AB8000086BFF1FBA46FF1FB046FF1F4046FF1F5E
:10AB90006846FF1F8846FF1F030010B50020DB0733
:10ABA00004D50721024A034800F08CF810BDC046C6
:10ABB00010C200114046FF1F054A0300106800281C
:10ABC00003D082889A4201D1806870470068F6E716
:10ABD000246DFF1F0A88030008009A4204D08A8867
:10ABE00004309A4200D0002070470000F8B5F822E7
:10ABF00000230D4F0D4E7968050042433370994292
:10AC000000D07B600A4C0021200000F011FF0023DF
:10AC10001A007C60AB4202D100203370F8BD0133D2
:10AC20002280DBB2F834F5E7246EFF1F206EFF1F91
:10AC3000286DFF1F73B56B4601900600684615002E
:10AC40001980FCF75FFF041E11D1002D0FD076890B
:10AC5000002E11D00C2000F04BFF00280ED0084A27
:10AC60000460136886808560002B02D1106020008C
:10AC700076BD1A001B68F7E70224F8E71324F6E70D
:10AC8000246DFF1F012100220A4B10B549420A4CD6
:10AC9000198099809A719A70084B20700120198050
:10ACA0005A60FFF7A3FF2078FCF78AFF0448FDF7FE
:10ACB00045FF10BD286BFF1F2C6EFF1F246EFF1F6A
:10ACC00071AD0011022310B5002802D0FFF7B2FFCA
:10ACD0000300180010BD0000030010B50020DB07C2
:10ACE00004D50421024A0348FFF7A4FF10BDC04663
:10ACF00024C20011C046FF1FF0B50E2687B0039393
:10AD00000CAB1F8802ABF618050008003100029258
:10AD1000FDF77AF804000120002C0FD03088FFF7EF
:10AD20004BFF03000E20002B08D05E68002E05D0DC
:10AD300021002800039B029A0097B04707B0F0BD9E
:10AD40000A4B10B5984207D10122002352420A80D3
:10AD50008B708A808B7110BDFFF73CFF0028FAD002
:10AD600001235B42038000238370F4E7FFFF0000B0
:10AD7000F8B5050001290AD1134E00243388F827BD
:10AD8000AB4219D028001149FFF7DAFF06E002298B
:10AD900004D10139FDF750FF0028EDD0F8BD3B008C
:10ADA00063437268D018D35A002B09D03A000021AF
:10ADB00000F03EFE0134E4B2054B1B78A342EED80E
:10ADC00001235B423380DDE7246EFF1F286BFF1FEA
:10ADD000206EFF1F10B5FFF7FDFE03000020834229
:10ADE00000D0987810BD0000F0B589B01C000EAB03
:10ADF00080CB03901E8810AB1B78049202930B7AD1
:10AE00000D00DB0616D42B780593022B24D0049872
:10AE1000FFF7D2FE002812D003689C46002B0ED00C
:10AE2000029B2200019329003B0064460398009690
:10AE3000A04705E00498FFF7BFFE002802D10E20CE
:10AE400009B0F0BD8368002BF9D00A2229000398CD
:10AE500098470028D7D0F3E76B6858781A786B4B7F
:10AE6000000210439842D2D8043B984210D2684B5B
:10AE7000984242D015D8674BC0180128C7D80B207C
:10AE8000002EDDD1EB681A7859683A80200028E05E
:10AE9000614BC018032800D979E000F009FD846AED
:10AEA000789E5E4B9842B2D10B20002EC8D1012370
:10AEB0003B80EB6831001B7823706889013080B2D9
:10AEC000FCF7A2FF3A88031E0ED0017802328A18DE
:10AED0003A80428962704289120AA27059680278E7
:10AEE000E01C00F09DFF06E004323A8031000422AD
:10AEF000601C00F09DFD0020A2E70B20002E9FD1DA
:10AF0000EB6807A91E8804233B80330A30002670B3
:10AF10006370FCF779FF051E28D004AB9A890E23D5
:10AF200004A95B183E49C668FCF7E2FF00280BD174
:10AF30002B783C486A680599FBF798FB002803D1F9
:10AF4000012304AA5B42D3813278022A06D17168B8
:10AF5000201D00F065FF3B8802333B800E2304AACE
:10AF60009B181B88A3701B0AE370C4E704ABDE8147
:10AF7000F4E70B20002E00D062E7E9680398FFF7A2
:10AF800029FF02233B802070000A6070B3E70B208A
:10AF9000002E00D054E70222EB681B883A80237011
:10AFA0001B0A6370A7E7E86800F0D2FCC2B2030096
:10AFB0000720B24200D243E70DD00299DBB27118EC
:10AFC000994202DB921BD3B20293029BE9681A00FA
:10AFD0003B8089195AE70023F6E70B20002E00D0AA
:10AFE0002EE70722EB683A801A7822705A7862704E
:10AFF0005A88A2705A88120AE2701A792271DA8885
:10B000006271DB881B0AA37175E7C0460429000042
:10B010000228000000D8FFFFFFD6FFFF0328000032
:10B02000FFFF000054C10011F0B58DB06B46002049
:10B03000089120229B5E83423DDAA64B187800F0EF
:10B04000F7FD071E32D00378B02B2CD100790238DF
:10B0500016281FD800F00CFC17001E001E001E0052
:10B0600031001E0096001E001D011E0052011E0030
:10B0700073011E00CD011E0050021E001E001E00A6
:10B080008E021E00E302944B94491B8878880B8043
:10B09000FBF72CF83800FCF7ADFF914B1B68002B39
:10B0A00001D038009847380000F0B2FC8020089B9F
:10B0B0000002434018000DB0F0BDF6220021874881
:10B0C00000F0B6FC0BAA3B7B7989388900923A00E4
:10B0D0000D32FCF7B1FD0400804B1B78002C3FD1F2
:10B0E00046E0804B788805937F4B4100CB5A0BAEEE
:10B0F000073BDBB232880293002301937B4B210094
:10B1000006930093059BFFF76FFE744D002810D146
:10B11000069B3A8A1B889A420BD138000599123057
:10B1200000F096FB002804D02B7862899B00EB1876
:10B130005A80162306A81B18328820007989FCF74C
:10B14000D7FE2B7804009A00AA1851880029C3D092
:10B150000133DBB22B70002807D006A9C98A918081
:10B16000634A12889A42BCD802E001214942918088
:10B17000002B04D059497888FAF7ECFF8AE73E891A
:10B180000A2479E000253E89574B06937B88069A6E
:10B190005B009B5A033B9D4202DB002DF0D05BE03D
:10B1A000162206A812183B7B798900923A003000DB
:10B1B0000D32FCF741FD0590002858D04689017AF0
:10B1C0007888FCF703FD041E44D1464B788807932A
:10B1D000069B4100C95A454B0439C9B206AAD28A16
:10B1E00006930291019400930599079BFFF7FCFDDC
:10B1F000041E2FD1069B39491A88931C002D26D195
:10B200004B807988384B4900CB5A5119033B8B420C
:10B2100020DD059B31485B8941190B71A91C013563
:10B22000C9B2EDB2059145191B0A2B71059B2D4939
:10B230000433181800F0F4FD2C4B059A1B88D31822
:10B24000DDB22C4B9E4205D00136B6B29CE7498850
:10B250009942D6D0002D0CD0204C2800618800F0F7
:10B2600007FE207021007888FAF784FF12E7059C1A
:10B27000F0E7002C00D183E77B78142B00D109E79D
:10B2800016493B794E800B700C717888FAF724FFD1
:10B2900000E7162406ABE41821003889FCF7B4FD5A
:10B2A000011E00D1B7E1788822880F4C45002C5B45
:10B2B0000A4D013CE4B2029400240F4B0194009526
:10B2C000FFF792FD041E00D014E129007888FAF7F8
:10B2D00061FFDFE62C6EFF1FAC45FF1F306BFF1FC9
:10B2E000246BFF1F2A6CFF1F6067FF1F206DFF1F6D
:10B2F000AA45FF1FFFFF0000326BFF1F162406AB9D
:10B30000E41821003889FCF77FFD011E00D182E19D
:10B3100078882288AE4C45002C5BAE4D013CE4B2EF
:10B3200002947C89AC4B01940095FFF75DFD041EEF
:10B3300000D0DFE029007888FAF736FFAAE600257A
:10B34000A44B1D803B00FE331B78A24A78880792ED
:10B35000AB4208D99E4B12880693069943005B5A6C
:10B36000013B9A4203DB0799FAF728FF92E616247D
:10B370006B00FB18059306ABE418059B21001889A8
:10B38000FCF742FD011E03D1059B01241E8973E7D2
:10B390007888924B2288069C099343001B5B904E51
:10B3A000013BDBB20293002300960193099BFFF758
:10B3B0001BFD041E02D0059B1E895DE77B88069A53
:10B3C0005B009B5A079A108832881218934202DC5D
:10B3D0001B1A013B33807F4C0230328809990019D7
:10B3E00000F01EFD2388328801359B182380EDB2C2
:10B3F000A8E70BAA3B7B7989388900923A000D3285
:10B40000FCF71AFC00250590059B002B04D10A24AB
:10B41000002D00D16EE060E0059B7888197AFCF77A
:10B42000D5FB0100041E63D1694C6C4B78880694EF
:10B430000993069B4400E45A694B063CE4B20BAE08
:10B44000328807930294019100930599099BFFF7B5
:10B45000CBFC041E4CD1079B5E491B881A1D002D96
:10B4600030D14A80059B5B4C5A8963191A716B1C59
:10B470009BB2E318120A1A71162306A832881B1809
:10B4800079890598FCF734FDFF21AA1C2E1D033590
:10B490000B00059092B2B6B2ADB2002803D006AB55
:10B4A000DB8AD9B21B0AA218651911712B714C4D98
:10B4B000301D2A884949201800F0B2FC2B88F61864
:10B4C000B5B2A1E74988914207D17A88069952001E
:10B4D000525AEB18053A9A42C4DC3E4C2800618867
:10B4E00000F0D6F9207021007888FAF771FED1E5D6
:10B4F000002DF2D13E89BFE6162606ABF6183100C4
:10B500003889FCF781FC3D000400FF3500282DD070
:10B51000037A9B060CD400227B89398978880092B3
:10B520003A000C32FFF7E8FB041E10D03E8915E00C
:10B530003088FFF741FB00281AD08368002B17D012
:10B540002100122278889847041EE4D0EEE7AB78F9
:10B55000002B02D17888FAF74BFE0026AB78002B3F
:10B5600000D097E5002C00D194E585E60124DDE7C5
:10B570000E24DBE7162506ABED1829003889FCF709
:10B5800043FC041E47D0037A9B0611D4154A7B88DE
:10B590001188994203D01448814207D11380134B7C
:10B5A000F8261D780023D9B2A94221D30924A1E7A6
:10B5B0002888FFF701FB00282FD08368002B2CD0B0
:10B5C0002100122278889847041EDFD092E7C046F7
:10B5D0006067FF1F306BFF1F326BFF1F2A6CFF1F5E
:10B5E000206DFF1F246EFF1FFFFF0000206EFF1F56
:10B5F00031005943546801336018615A0029D2D18F
:10B600003C0008342100F82200F00AFC2100788870
:10B61000FAF7F6FD3EE501246CE70E246AE71D4BC0
:10B620001A887B889A4231D07888FAF7F3FD31E5A1
:10B63000F823059851684343CD18C95A00291FD0F3
:10B640003B7A012B0BD16C88AB887888AA1D0094BB
:10B65000FFF752FB041E02D000233B722E88F82213
:10B660000021280000F0E4F900232B80059B013322
:10B67000DBB20593084B05991B78064A8B42D7D855
:10B6800001235B421380002CCED0F5E50026340068
:10B690000596EFE7246EFF1F206EFF1F70B50400B4
:10B6A0000E001500FFF796FA031E08D13100054879
:10B6B000FFF790FA03001120002B02D01C8000201D
:10B6C0009D7070BDFFFF0000F8B50B4F06003B7882
:10B6D0000D001400FF2B0ED00A2000F091F9011E7E
:10B6E00009D0B1230380002346800371C580048103
:10B6F000387800F055FAF8BD0147FF1FF7B50F0085
:10B7000008A90600088809A90B240988002821D166
:10B710000234022B1ED1557813782D021D432B00C5
:10B720008B4301937334002B14D1FB683000190054
:10B730000093FFF74FFB019C85420BD02A0030009D
:10B740000099FFF7ABFF041E04D12A00300079896D
:10B75000FFF7BAFF2000FEBDF0B50E7885B003906C
:10B760000AA805880120022E0DD14C68277864783C
:10B7700024023C43054FBC4205D10398DBB201963D
:10B780000095FFF7BBFF05B0F0BDC04602290000E1
:10B7900010B504000C4800F053FA0C48A16B00F0FF
:10B7A0004FFA0B48E16B00F04BFA0A48216C00F0AD
:10B7B00047FA094B0948196800F042FA084B1B6820
:10B7C000002B00D09847FEE7E6BF0011FCBF001138
:10B7D0000BC000111AC0001104ED00E029C00011D7
:10B7E000306EFF1F002307B501A80193FFF7D0FFBC
:10B7F000044A0548002110B5121A00F019F9F8F7AB
:10B80000DFF8FEE7346EFF1F0447FF1F0000000053
:10B8100001B40248844601BC604700BF45500000A7
:10B8200001B40248844601BC604700BFC94A010018
:10B8300001B40248844601BC604700BFF30E00001B
:10B8400001B40248844601BC604700BF6D30FF1F51
:10B8500001B40248844601BC604700BFCD4C0100E2
:10B8600001B40248844601BC604700BF7D18FF1F39
:10B8700001B40248844601BC604700BFD93DFF1FA8
:10B8800001B40248844601BC604700BF6DBC0000A3
:10B8900001B40248844601BC604700BF090E0000A5
:10B8A00001B40248844601BC604700BFD91B0000B8
:10B8B00001B40248844601BC604700BFC53DFF1F7C
:10B8C00001B40248844601BC604700BF0D5201002C
:10B8D00001B40248844601BC604700BF014C01002E
:10B8E00001B40248844601BC604700BFD53AFF1F3F
:10B8F00001B40248844601BC604700BF55220000E5
:10B9000001B40248844601BC604700BFB930FF1F44
:10B9100001B40248844601BC604700BF9D32FF1F4E
:10B9200001B40248844601BC604700BF055E0000C8
:10B9300001B40248844601BC604700BFC534FF1F04
:10B9400001B40248844601BC604700BF017F00008B
:10B9500001B40248844601BC604700BFDD520100CB
:10B9600001B40248844601BC604700BFC51D000009
:10B9700001B40248844601BC604700BF5D32FF1F2E
:10B9800001B40248844601BC604700BFED4A010093
:10B9900001B40248844601BC604700BFC95C010095
:10B9A00001B40248844601BC604700BF0124000086
:10B9B00001B40248844601BC604700BF3938FF1F0C
:10B9C00001B40248844601BC604700BF8D120000EC
:10B9D00001B40248844601BC604700BFC53F000077
:10B9E00001B40248844601BC604700BF291C000026
:10B9F00001B40248844601BC604700BFE532FF1F26
:10BA000001B40248844601BC604700BF1D4D0100DF
:10BA100001B40248844601BC604700BF434D0100A9
:10BA200001B40248844601BC604700BF0D3CFF1FC3
:10BA300001B40248844601BC604700BF154D0100B7
:10BA400001B40248844601BC604700BFC92600001B
:10BA500001B40248844601BC604700BF8552010022
:10BA600001B40248844601BC604700BF595201003E
:10BA700001B40248844601BC604700BFADAE00007F
:10BA800001B40248844601BC604700BF0189000040
:10BA900001B40248844601BC604700BF311B00006E
:10BAA00001B40248844601BC604700BF4532FF1F15
:10BAB00001B40248844601BC604700BF151BFF1F4C
:10BAC00001B40248844601BC604700BFC9A9000018
:10BAD00001B40248844601BC604700BF5D17000006
:10BAE00001B40248844601BC604700BF1147010011
:10BAF00001B40248844601BC604700BF3D4B0100D1
:10BB000001B40248844601BC604700BF8B5201006B
:10BB100001B40248844601BC604700BFB70E000074
:10BB200001B40248844601BC604700BFC521000043
:10BB300001B40248844601BC604700BFF535FF1FD1
:10BB400001B40248844601BC604700BF213BFF1F8F
:10BB500001B40248844601BC604700BF2D38FF1F76
:10BB600001B40248844601BC604700BFB54C0100E7
:10BB700001B40248844601BC604700BF8534FF1F02
:10BB800001B40248844601BC604700BF252600007E
:10BB900001B40248844601BC604700BF810E00002A
:10BBA00001B40248844601BC604700BF594F010000
:10BBB00001B40248844601BC604700BF4551010002
:10BBC00001B40248844601BC604700BF156B010008
:10BBD00001B40248844601BC604700BF4D1F00000D
:10BBE00001B40248844601BC604700BFA54F010074
:10BBF00001B40248844601BC604700BFA946010069
:10BC000001B40248844601BC604700BFA13BFF1F4E
:10BC100001B40248844601BC604700BF091B000014
:10BC200001B40248844601BC604700BF75A900000A
:10BC300001B40248844601BC604700BFF54E0100D4
:10BC400001B40248844601BC604700BFE53A0100E8
:10BC500001B40248844601BC604700BFC56D0100C5
:10BC600001B40248844601BC604700BFE1170000F0
:10BC700001B40248844601BC604700BF456B010027
:10BC800001B40248844601BC604700BFB3520100C2
:10BC900001B40248844601BC604700BF5549010019
:10BCA00001B40248844601BC604700BF9DA9000062
:10BCB00001B40248844601BC604700BFE54800006B
:10BCC00001B40248844601BC604700BF1D4B01001F
:10BCD00001B40248844601BC604700BFB14E000079
:10BCE00001B40248844601BC604700BF893CFF1F85
:10BCF00001B40248844601BC604700BFF94C010012
:10BD000001B40248844601BC604700BF5118FF1FC0
:10BD100001B40248844601BC604700BF851F000093
:10BD200001B40248844601BC604700BFE139FF1FEF
:10BD300001B40248844601BC604700BF2D39FF1F93
:10BD400001B40248844601BC604700BFEDA5000075
:10BD500001B40248844601BC604700BF5D38FF1F44
:10BD600001B40248844601BC604700BFB13DFF1FDB
:10BD700001B40248844601BC604700BF090E0000C0
:10BD800001B40248844601BC604700BF2124000082
:10BD900001B40248844601BC604700BFE93AFF1F76
:10BDA00001B40248844601BC604700BF350E000064
:10BDB00001B40248844601BC604700BFB53CFF1F88
:10BDC00001B40248844601BC604700BF35550000FD
:10BDD00001B40248844601BC604700BF79180000E6
:10BDE00001B40248844601BC604700BF51470100CE
:10BDF00001B40248844601BC604700BF51250000E1
:10BE000001B40248844601BC604700BF056A0000D7
:10BE100001B40248844601BC604700BFDD660100F2
:10BE200001B40248844601BC604700BFE94C0100F0
:10BE300001B40248844601BC604700BFD9490100F3
:10BE400001B40248844601BC604700BF3D180000B1
:10BE500001B40248844601BC604700BF295101007B
:10BE600001B40248844601BC604700BF657101000F
:10BE700001B40248844601BC604700BF350E000093
:10BE800001B40248844601BC604700BF691F00003E
:10BE900001B40248844601BC604700BFE9280000A5
:10BEA00001B40248844601BC604700BF613BFF1FEC
:10BEB0000003010302020302040205000602070058
:10BEC000080009020A030B030C000D000E030F0308
:10BED00010031103120313001400150316030000CE
:10BEE000BD3D0011F13D0011000000000200000006
:10BEF000F6BE0011192A0F1809000000F1590000C0
:10BF0000FD2400004582001159A20011AD760011F8
:10BF100049800011B554001129B000111D510011C4
:10BF2000AD3F0011DD4000110000000016160000BA
:10BF3000020000003CBF0011F4FFF3FFD2FC000040
:10BF40001D420011000000000000000054757961DE
:10BF50000042312E33003030313800676974687523
:10BF6000622E636F6D2F70767678005448303500FE
:10BF70000200000084BF0011292A282A272A262A25
:10BF8000252A242A0A180000E20400007102000099
:10BF900078EC0000744000001027000060F0000002
:10BFA00006640000204E00000000000005000000B4
:10BFB0001F501D00023CB4000001180013000000D7
:10BFC000A10200003031323334353637383941423E
:10BFD00043444546005048592B36325858504C552A
:10BFE0005330353034005B48617264206661756C93
:10BFF000742068616E646C65725D0A004C5220208A
:10C00000203D203078253038780A00504320202009
:10C010003D203078253038780A0050535220203D9A
:10C02000203078253038780A0049435352203D208B
:10C030003078253038780A00B95800110D590011B0
:10C04000000000000200000050C000116F2A6E2A9C
:10C050001A18EAD8BC80F0FC600000000000000064
:10C0600000005F066B2F363D7D077F3F777C596E62
:10C070007971AF066D4FC6CBEB0EEFCFEEC3A9665D
:10C08000E9E8FA60D6F46CBCBEE0FEFCEE3E9A76BF
:10C090009E8E000001A00000000000006410B71D8B
:10C0A000C8206E3BAC30D9269041DC76F4516B6BE6
:10C0B0005861B24D3C7105502083B8ED44930FF0A8
:10C0C000E8A3D6D68CB361CBB0C2649BD4D2D3865E
:10C0D00078E20AA01CF2BDBDFB349B5F80000080AB
:10C0E0000010000000000000AF620011397900115B
:10C0F000D3620011417D001157630011177D0011BB
:10C10000CD630011ED7C00111F640011B57E00119C
:10C1100087640011B57E0011B96400116F7E0011B3
:10C12000CD630011A57C0011456400114D7E001106
:10C1300000000000000000002B6500114D7E001182
:10C140008D65001151790011052A042A012A002A5F
:10C150000229032801280028011800180000000007
:10C160000000000000000000000000870101020143
:10C1700002010102010203030401030101010101A3
:10C180000303020103000D000E0010001100130054
:10C190001401070108010A010B011C011D02040220
:10C1A00005020702080219021A021C021D030103FC
:10C1B000020317000201000504000807000B0A0033
:10C1C0001716001D1C010201010504010E0D0111CD
:10C1D00010011413011716011A19020201020B0AA9
:10C1E000020E0D02111002141302171603050403A8
:10C1F0000807030B0A030E0D0001020307090A0BCF
:10C200000E0F101112141718191A1B1F20212200CB
:10C2100071A900112DAA0011000000000200000009
:10C220005AC100110000000059B7001100000000C1
:08C230000200000058C10011DA
:020000041FFFDC
:1000000000000000193F0011FCBE0011F8BE0011F5
:100010001064FF1F0000000000000000000000004E
:1000200000000000000000000000000000000000D0
:1000300000000000000000000000000000000000C0
:1000400000000000000000000000000000000000B0
:1000500000000000000000000000000000000000A0
:100060000000000000000000000000000000000090
:100070000000000000000000000000000000000080
:100080000000000000000000000000000000000070
:100090000000000000000000000000000000000060
:1000A0000000000000000000000000000000000050
:1000B0000000000000000000000000000000000040
:1000C0000000000000000000000000000000000030
:1000D0000000000000000000000000000000000020
:1000E0000000000000000000000000000000000010
:1000F0000000000000000000000000000000000000
:1001000000000000000000000000000000000000EF
:1001100000000000000000000000000000000000DF
:1001200000000000000000000000000000000000CF
:1001300000000000000000000000000000000000BF
:1001400000000000000000000000000000000000AF
:10015000000000000000000000000000000000009F
:10016000000000000000000000000000000000008F
:10017000000000000000000000000000000000007F
:10018000000000000000000000000000000000006F
:10019000E934FF1F3133FF1FC1660100000000007A
:1001A000000000000000000000000000000000004F
:1001B000000000000000000000000000000000003F
:1001C000000000000000000000000000000000002F
:1001D000000000000000000000000000000000001F
:1001E000000000000000000000000000000000000F
:1001F00000000000000000000000000000000000FF
:1002000000000000000000000000000000000000EE
:1002100000000000000000000000000000000000DE
:1002200000000000000000000000000000000000CE
:1002300000000000000000000000000000000000BE
:1002400000000000000000000000000000000000AE
:10025000000000000000000000000000000000009E
:10026000000000000000000000000000000000008E
:10027000000000000000000000000000000000007E
:10028000000000000000000000000000000000006E
:10029000000000000000000000000000000000005E
:1002A000000000000000000000000000000000004E
:1002B000000000000000000000000000000000003E
:1002C000000000000000000000000000000000002E
:1002D000000000000000000000000000000000001E
:1002E000000000000000000000000000000000000E
:1002F00000000000000000000000000000000000FE
:1003000000000000000000000000000000000000ED
:1003100000000000000000000000000000000000DD
:1003200000000000000000000000000000000000CD
:1003300000000000000000000000000000000000BD
:1003400000000000000000000000000000000000AD
:10035000000000000000000000000000000000009D
:10036000000000000000000000000000000000008D
:10037000E5B70011000000000000000000000000D0
:10038000000000000000000000000000000000006D
:10039000000000000000000000000000000000005D
:1003A000000000000000000000000000951AFF1F80
:1003B000000000000000000000000000000000003D
:1003C000000000000000000000000000000000002D
:1003D000000000000000000000000000000000001D
:1003E000000000000000000000000000000000000D
:1003F00000000000000000000000000000000000FD
:081838004072FF1F4118FF1F61
:10184000024981F3088802F053FC00004072FF1F38
:1018500010B502F005FB072804D0122808D0022892
:1018600008D010BD044A0420136B01331363F8E75A
:101870000220F6E71420F4E70868FF1FF8B5070018
:101880000C0026002500503630785135002804D150
:101890000300287058342370F8BD2978CA00481E08
:1018A0008141A3183800A25C5B68C9B2FFF7D0FF82
:1018B00000280DD12B78DA00A218013350602B706C
:1018C0003378044A013B3370136A01331362D8E75B
:1018D0000123DFE70868FF1F5C234343074910B576
:1018E000C9180B0058331B78012B05D1FFF7C6FF31
:1018F000034A936A0133936210BDC0463C68FF1FE0
:101900000868FF1F10B502F033FC064A01211300DE
:1019100010CB4942D967044B136002F0D9FA20007A
:1019200010BDC04600E100E01000100010B504003A
:1019300002F01EFC024B1C6002F0CAFA10BDC04649
:1019400000E100E010B5040002F012FC4021094A59
:10195000200013688B43136002F08AFB01F0A6FDA0
:101960000022054B01201A60044B04321A6002F079
:101970001FFCFEE71CF00040C4F00040C0F0004037
:10198000431E5A425341A022F0B5D2015B4213409C
:10199000154D164A40019B182A18127E8BB00191F2
:1019A000002A1BD01A000832D46F0022E6B206AF1C
:1019B000E4B294420EDC2818C369002B08D00199C8
:1019C00002AA117106AA049202AA167303A89847E4
:1019D0000BB0F0BD1978B9540132EAE71A7D1A78D4
:1019E00006AB01261A70E6E7C86AFF1F00400040F8
:1019F000F0B5254B04004001C25C85B0002A2BD015
:101A00001A18117E002927D0917E002924D011793F
:101A1000022921D11689D788D168F51BADB22A1CBD
:101A2000102D00D9102292B2BE4217D118180123EE
:101A300003710023C269C38003819A4206D06846BD
:101A4000032103730171029301A890470820002C21
:101A500000D0192001F022FC05B0F0BD013C654228
:101A60006C41A0256442ED012C40084D1B186419FF
:101A7000074D0633013A92B2AA42EDD01888461CAF
:101A80001E80085C2070F5E7C86AFF1F0040004018
:101A9000FFFF00000F220E4B10B59868104002386F
:101AA0000A280BD802F08EF90D0A0B0A0A110A0A4D
:101AB0000A0A060002210020FFF762FF10BD012183
:101AC000F9E70020FFF794FFF8E7DB6FF6E7C04681
:101AD000004000400F220E4B10B5986810400238AD
:101AE0000A280BD802F06EF90E0A0B0A0A120A0A2B
:101AF0000A0A060002210120FFF742FF10BD012162
:101B00000800F9E70120FFF773FFF7E7DB6FF5E760
:101B10000090004013B5334C2378072B3DD8324B4F
:101B20001A78324B002A39D18022196852020A43AE
:101B30001A60252001F0F4FF20232D4A11680B4381
:101B4000802113606B460422C905086807331042E0
:101B500028D080210422C905C86810422ED08021D7
:101B60002020C905CA688243CA6014221A701A78F4
:101B7000002A2FD18021C905C86820320243CA60DB
:101B800014221A701A78002A28D11A4B1A7D22784A
:101B90005A601D221A705932DA6013BD1A6816494C
:101BA0000A40C5E7086802430A6014221A701A78CE
:101BB000002ACED01A78013AD2B2F7E7C8680243B9
:101BC000CA6014221A7019784A1ED2B21A700029FB
:101BD000F9D1C4E71A78013AD2B2C7E71A78013AC4
:101BE000D2B2CEE73C46FF1F0447FF1F3CF0004047
:101BF0003446FF1F00200040FFFFFEFF564B70B52C
:101C00001B68012B03D1554A936D0133936502F094
:101C1000FFF9534B534A1860534B544C1A6001233D
:101C2000534A1360534A13602378002B06D00622D0
:101C30005149524802F02CF900232370504A514B6D
:101C400010681B78C1B2002B0ED14F4CC0B2237864
:101C50005BB2002B4FDB237824785BB264B21B04A9
:101C600024021B191B1813600B1C50294ED950233A
:101C7000464A47491078DBB2FF2202284BD1086858
:101C8000444C454D267890432A78964254D9227880
:101C900024782E78023B5D10A31B6B435201D31AAC
:101CA00010335B111843086002F002F9031F012B87
:101CB00045D83A4B1B78002B06D0394B1B78002BAC
:101CC00002D0002002F054F9A122364B92009978FC
:101CD000354B4A431B689B18832292009B181B7844
:101CE000033B012B03D8AF20400002F0C1FA0122D0
:101CF0002E4BDA8270BD237824785BB264B2FF3356
:101D0000FF341B0424021B190138ABE7CAB2022AB4
:101D1000AED20223ACE70868254C264D26789043C6
:101D20002A78964208D9227824782D78023B5B10D5
:101D3000641B63435201B2E72378DBB2B2E70228A7
:101D4000D5D11D4B1B78013B022B03D91B4B1B78B4
:101D5000022BCCD16C20C8E79809FF1FFC0FFF1F96
:101D60004067FF1FFF3F0000141003404467FF1F40
:101D70000C10034000100340D50BFF1F7211FF1F12
:101D8000B40003408C09FF1F680AFF1F490AFF1FA8
:101D900094000340460AFF1F470AFF1FF908FF1F70
:101DA0002209FF1F300DFF1F3409FF1FBC0BFF1F4F
:101DB000440AFF1F450AFF1F1C09FF1F2309FF1FBD
:101DC00010B502F025FA0022014B1A8010BDC04662
:101DD0003C67FF1F10B502F073FAA121054A890084
:101DE0009478054A61431268044B5218528C1A8049
:101DF00010BDC046300DFF1F3409FF1F3C67FF1F99
:101E000010B50D4B0D4A9978A1239B004B431268E6
:101E1000D218531DD97F0A4B1B88994209D2441C02
:101E200007D0C82805D0D2695B1A5A43054B5343E3
:101E3000C01802F0E5F910BD300DFF1F3409FF1F77
:101E40003C67FF1F7102000070B5244D2B68002B0A
:101E500028D002F085F82B68D8402B680400002BAE
:101E600027D002F00DF92B68D8401D4B1D4A9978F8
:101E7000A1239B004B431268D118D25C91239B0095
:101E8000002A20D0CA580132CA50174B17491B6884
:101E90000868834214D3D23B181A012A1AD0144B73
:101EA000186070BD02F05CF8124B196802F078F906
:101EB000D3E702F0E5F80F4B196802F071F9D4E7A7
:101EC0000D495B18E8E7CA500C4B1B68DB68E41847
:101ED000201AE4E7F530FF30E1E7C0461C08FF1F99
:101EE000300DFF1F3409FF1F9C09FF1F4067FF1FB4
:101EF000A009FF1F1808FF1F2DFF3F004867FF1FA5
:101F000070B504000D00282916D10300A433C2883F
:101F10001B889B1A0B4A9BB293420DD906006A3666
:101F200005223100653002F063F9002804D1310048
:101F3000200002F00DF870BD2900200002F038F8F2
:101F4000F9E7C046FE7F0000F8B50400012002F06A
:101F5000A7F902F0BDF9174A17491060174D0300A1
:101F6000886A174E28607568AC46164D2F680025A4
:101F7000BC4501D275687D1B134E00193560C862DF
:101F8000A4204C6A40032043486210490978002984
:101F900005D00F490978022902D10F3B1360F8BD23
:101FA000012901D1083BF9E7032901D1053BF5E7F8
:101FB000033BF3E7E408FF1F00F00040340AFF1F73
:101FC00028100040180AFF1F1C0AFF1F1C09FF1FD2
:101FD0004A0AFF1F70B580241025E405A3682B432F
:101FE000A36002F02DF9A368AB43A36070BD0000AD
:101FF000F7B5160080221C001023D20501919168CC
:1020000005000B43936000225A4BD7301A6001F051
:10201000EFFF9D232A002F009B00EB58CA320121BD
:102020000092FC37002B01D00021009A386801F0A3
:10203000C7FF2900009BCB311A784F4BD3351A606C
:102040004B780A781B0213438A7812041A43CB7820
:102050001B061343494A1BBA13604B790A791B02CA
:1020600013438A7912041A43CB7931001B061343B8
:10207000434A1BBA13606B782A781B021343AA7871
:1020800012041A43EB781B0613433E4A1BBA136033
:10209000019A330213433C4A13603C4B22001B1B42
:1020A0009C4603293DDCB3089A0013005142B21A42
:1020B000032A46D1354AE018511A82784078120432
:1020C00000020243E05C043302430A600022FF2B5B
:1020D0004BDDF0222E4B12011A600F222D4B1A609D
:1020E0002D4A1368002BFCD00023224A2749136095
:1020F000091B321D0B191B68043A180A2370607003
:10210000180C1B0EA070E3700434002AF2DC80224D
:1021100010213B68D20501333B6093688B43936089
:10212000F7BD6346D578981893782D061B042B438A
:10213000157804392B43557804322D022B43036064
:10214000AFE7022A0AD1114AE05C511AE21852782C
:10215000120202430A6004339BB2B7E7012AB5D1E9
:102160000A4A521AE15C1160F5E7084959180A60F9
:102170000433ACE7000004403C0004403800044055
:1021800034000440300004400C00044000010440CE
:10219000040004401000044014000440F7B515008A
:1021A00080221C001023D2050091916807000B4388
:1021B00093600023654AD730136001F019FF9D2317
:1021C0003E009B00F9583B00CA363200FC33002920
:1021D00000D07FE0586801F0F3FE390032785C4BA4
:1021E000CB311A604B780A781B0213438A78AC46CD
:1021F00012041A43CB78281D1B061343554A1BBAF9
:1022000013604B790A791B0213438A7912041A432B
:10221000CB791B061343504A1BBA13604B7A0A7AD8
:102220001B0213438A7A12041A43CB7A21001B063D
:1022300013434A4A1BBA1360009A2B021343484ABD
:1022400013602200474B1B1B0093009BCE785B184A
:1022500001938B7836061B0433430E7804383343DE
:102260004E78043136023343019E33600328ECDCA0
:102270000321A808431C9B002940800003292BD17F
:102280003849E5185E18A9786D78E35C09042D02D9
:10229000294319433160030008330021FF2B2DDD52
:1022A000314B324919600F21314B19600123274905
:1022B0000B60304B19680029FCD006211B680B40CD
:1022C000042B20D080220020D20593680A318B4352
:1022D0009360FEBD01217DE7022908D121495D18E7
:1022E000E1184978E35C090219432960D3E7012921
:1022F000D3D11C495918E35C0B60CCE71948181876
:1023000001600433CAE7002310490B606346002BC9
:102310000CDC3B00FC335A68102101325A608022E9
:10232000D205936801208B439360D2E7009B9B18F2
:102330001B68190A13705170190C1B0ED3700423FB
:102340005B4291709C440432E0E7C04600000440C8
:102350003C00044038000440340004403000044095
:102360000C0004400001044004000440080F000079
:10237000100004401400044070B5061E19D002225B
:10238000614B9B799343012B13D1604B1A78FF2A41
:102390000FD15A78FF2A0CD19A78FF2A09D1DA781E
:1023A000FF2A06D11A79FF2A03D15B79FF2B00D1CE
:1023B000A7E0574B0C201A78012A08D00022554D6F
:1023C0001A702B781A00093A042A01D8212070BD0E
:1023D0005A1F012AFAD94C4CA07B042800D990E05E
:1023E000A279032A00D98CE0821E012A03D86288D0
:1023F0001F2A00D885E0002E61D0012E00D080E099
:10240000A288012AE2D0002B0AD10138032803D880
:1024100001F0D8FC151D19151F202E7001F0B8FE13
:102420002B785A1E032A16D800253B4B1D60282303
:10243000237501F00DFFA8422ED0A580C6E7022328
:1024400020202B70EAE7042322202B70E6E70323E9
:1024500021202B70E2E7073B012BB7D82F4B1B68DD
:10246000DB6A9B06B2D52E4B1A78002AAED1A27B2E
:10247000911E012901D9002AA8D1022280211A70B7
:102480002823284D89012878237501F089FD8021B2
:102490002878890101F0E4FD0123A380224B1B78F9
:1024A000002B0AD0FA228021204B92001B880902BF
:1024B0005A431C4B187801F0DBFC002087E701F041
:1024C00057FE2B78A680073B012B06D918482E70A3
:1024D00001F006FF1E2001F05BFE114B114C1A7833
:1024E000002A06D080210022207889011A7001F08C
:1024F00057FD01F0EDFC80212078090201F050FD2C
:10250000DBE7122063E7C046A60BFF1F6B09FF1F26
:102510001A09FF1F1C09FF1F4809FF1F4867FF1FFB
:102520002309FF1F1B09FF1F2109FF1F2C09FF1F84
:102530000010004010B5002901D001F021FE10BDAF
:10254000F7B5604B01919978A1239B004B435E4AFC
:10255000060014681022E418D6235B00E0583623E6
:10256000FF33E35C00279343222B41D1574B0F3AB3
:102570001A600760012501F093FD019B1880E82394
:102580005B00E35C002B01D0B34258DD0023504FC9
:10259000FB70AD33FF33E3581A68002A03D09B88E1
:1025A000DB439B071DD03823FF33E35C002B18D09F
:1025B0009B235B00E35C002B13D1D133FF33E35C3F
:1025C000B3420EDAA4235B00E15AE018090A023193
:1025D00001F02EFD23000122FE33013E01351A8752
:1025E000FA70E8235B00E35C002B2AD0A8B2FEBDA2
:1025F00003683D00002BBED081880430090A0231F7
:1026000001F016FDD6235B00E3581F60B2E72300FC
:10261000B133BA00FF339858013781880430090A72
:10262000023101F005FDE8235B00E35CBB42EEDC18
:10263000E822F61AED1800235200A354A6E700275B
:10264000F1E7200001F0FCFB00281FD0002E1DDD6B
:102650007319882647190193B600200001F040FD48
:102660005A30800020184068013581880430090AFA
:10267000023101F0DDFC200001F0F2FDA35901332D
:10268000A351BD4202D0019B9D42E6D1114BE35CB8
:10269000002BABD095239B00E35C002BA6D00E4B08
:1026A000E15A0029A2D00D4AA35C994202D9013314
:1026B000A3549BE700231A212000A35401F090FDAE
:1026C00094E7C046300DFF1F3409FF1F001403407C
:1026D000E010FF1F5A020000720200005E020000BC
:1026E000F8B51D4B1D4F1A78002A10D1BA7B002A6D
:1026F00002D101321A7003E0032AFAD0022AF8D07C
:1027000001F0A6FD00220120154B1A70F8BD154BF3
:10271000154D1C68154B9E7801232B702878C0B28C
:1027200000F0CEFCBB7B002B0BD101F081FDA1237F
:102730009B007343E41883239B00E41823782B70D9
:10274000E4E7032B02D101F0CBFBF0E70020022BE2
:10275000DCD101F0B5FBEAE71C09FF1FA60BFF1F48
:102760002309FF1F3409FF1F490AFF1F300DFF1FF8
:10277000F0B587B00EAD2F780FAD2D780593AC4630
:10278000634614000E4D0CAA12782E7803930D9B0D
:10279000009201932200059B029701F0F9FB2E7035
:1027A000012C01D0042C08D1802206498B88934348
:1027B000054A1278D20113438B8007B0F0BDC046A2
:1027C0001C09FF1F6C11FF1F7809FF1F0B001B3B2B
:1027D00070B504003020E02B0DD81300E025493BF4
:1027E000FF3B9BB2ED00AB4205D8034B20001982A2
:1027F0005A8201F0A5FB70BD8410FF1F10B501F0D7
:1028000007FC054B00205B68052B04D9034A52687E
:10281000D20200D4980810BD00100040FCE100E096
:1028200070B501F0A5FC0D4B1B68FC33DC691D6A1B
:10283000FFF7E4FF6419844204D2094B01241B68AA
:10284000002B07D004220024064B1A70064A936915
:102850000133936101F03CFB200070BD4867FF1F0E
:102860009809FF1F2309FF1FFC0FFF1F70B50C4DB8
:102870002B68FC335C6A01F07BFCFFF7BFFF2B6821
:102880000025FC339B6AE318834204D2054B1B6886
:10289000AB4200D1051B01F01BFB280070BDC046F8
:1028A0004867FF1F9809FF1FD722044B92009B58CF
:1028B00010B5002B00D0984710BDC0460000FF1F88
:1028C000F0B587B001F008FAFFF7EEFFC54BC64C34
:1028D00004931B78022B45D1C44B1B68186A01F086
:1028E000DFFCC34BC34A1A60C34BC44A1A60A02220
:1028F000C34B52001A60049B187801F0D9FCC149FF
:10290000C14801F07DFBC149C14801F079FB1022AB
:10291000C04BFF201A60802252031A60802292036B
:102920001A60802212041A6001F022FB012001F0DB
:1029300057FBFA20400001F04BFB582001F098FCB7
:10294000B54801F075FA012001F0D2FC072001F032
:10295000AFFBE26DB14B1A4084235B001343E36588
:1029600007B0F0BD01F08CFAAD4E0290322001F0BC
:1029700097FC33681B0628D43C2001F091FC0F2003
:1029800001F08EFC974B1B78012B00D113E18025C1
:1029900033682B4200D0A1E0636C03202B436364B7
:1029A00001F07EFC01F06CFA029B0299C31A5A1ED8
:1029B000814200D81A009B4B1A608C4B19681E2369
:1029C0005343994A9B18CB618BE701F059FA802356
:1029D000E26BDB0213430390E363E26D8F4B032052
:1029E0001A4028231343E36501F05AFC0320A56E27
:1029F00001F056FCA36E0320DB03DB0B019301F017
:102A00004FFCA76EED03FF03ED0BFF0B874AAB18DE
:102A1000C22B2ED8019B9B18C22B2AD8BB18C22BC5
:102A200027D8019B2A009D4200D21A00019B9D429B
:102A300000D91D003B00974200D21300BD4200D9CF
:102A40003D005B1B122B14D80C22336814209343D7
:102A500033603368764A1340336001F021FC08216B
:102A6000A36EE26DDB038A43E265724ADB0B1360FF
:102A700085E7032001F014FCA36EDB03DB0B059359
:102A800001F0FEF9039B0399C21A531E814200D83C
:102A90001300694A93421BD9FF23356864492D0A04
:102AA0001D4032686B1C1B060A401B0C134333602D
:102AB0000C23326800209A43083B1343336001F033
:102AC0002FFC5E485E4BA840984205DCFEF73AFFBB
:102AD000019D0197059F99E75A48F7E700235A4E51
:102AE00033608023226CDB0213432364636C032076
:102AF0002B43636401F0D4FB3368013333608023DC
:102B0000626C5B021343636405230193E26D434BE4
:102B100003201A404D4B1343E36501F0C1FB08212C
:102B2000A26EE36D434F8B43E3653B6802394B4331
:102B3000D203D20B9A420CD89B1A3B2B0BD8E36DD5
:102B400043490B40E365636C0B406364414B1A607F
:102B500028E7D31AF1E7019B013BDBB20193002B7D
:102B6000D4D1E36D3A4A1340E365636C1340636468
:102B70003368042B07D9BFF34F8F374B374ADA60DE
:102B8000BFF34F8FFEE7636C0320AB43636401F038
:102B900087FBE26D214B03201A4028231343E36592
:102BA00001F07EFB0822A36EDB03DB0B3B60E36DD1
:102BB0009343E3659AE70722E36B1340012B02D1AD
:102BC000002001F075FB264D264AAB680220134019
:102BD000AB6001F065FB8023AA685B001343AB6028
:102BE000E0E6C0464A0AFF1F00F000404867FF1FAA
:102BF000000003400180063DBC0003403408000093
:102C0000A40003407102000014100040FFFF3F00C9
:102C10002810004000E100E03075000000FEFEFFDB
:102C2000C4F000403067FF1F7206000091FCFFFFF8
:102C3000FF00FFFF3867FF1FE30C0000E880000083
:102C40005F361E0060361E00A045FF1F28000100F1
:102C5000FFFFFEFF3467FF1F00ED00E00400FA05F0
:102C60003CF00040FFFEFFFF694E336888331B686D
:102C700083F3088801F05CFA00F018FC654B664AA3
:102C80001B68934207D0002001F04AFB0221634AEF
:102C900013688B431360FFF713FE614B614C187888
:102CA000C0B201F025F90023A3600233A3605E4B9C
:102CB0000120236001F0F4FA0323A36001F0E0F89F
:102CC000040001F0A5F9050001F0DAF8574B18608F
:102CD00001F01EFA564B1968621A531EA14200D227
:102CE00013008022D203934201D39B029B0A3268D5
:102CF000D16AC90700D478E04E491C0C09689BB220
:102D00004C4359432402090A641803274A49FC32F8
:102D100093680A6849489B1A494A4A4E12684A49C8
:102D20009B18414A34609A183B400193036892080B
:102D30009C46019B0A6063440360042B03D9013263
:102D40003B400A6003600B684049E418200001F032
:102D500027FA3F4F3D493B68C3183B602000019371
:102D600001F0AEF93B4C20680818384920608842D1
:102D700005D9019B01333B6001F0A2F9216001F00C
:102D8000BFF9354B1B78002B0ED001F041F93168AB
:102D9000324B4A1B1B6812189A4233D2591A4919EE
:102DA000091A2F4801F02CF92E4C237A002B0FD052
:102DB00001F02EF93168E3684A1B1218934224D9B6
:102DC000591A4919091A284801F01AF900232372DF
:102DD000264B83F3088801F03BF9022001F0D8F973
:102DE000002001F09DFA01F0EBF9DC0199000234BA
:102DF000641A5900641A09214B438033CB40A4085C
:102E0000E41882E7FA218900CBE71949DBE7C046DD
:102E10004867FF1F0C0AFF1FB64121031000004046
:102E2000490AFF1F14100040C4090000100AFF1FC8
:102E3000340AFF1F380AFF1F200AFF1F280AFF1F3E
:102E40001C0AFF1F2C67FF1F240AFF1F71020000CE
:102E50006008FF1F2C0AFF1F1C09FF1FE408FF1F4B
:102E600000100040740BFF1F3C10004000000020C9
:102E7000DC050000A022054B92009B5810B5002BEA
:102E800001D0984710BD01F0FBF9FBE70000FF1FE0
:102E9000A122054B92009B5810B5002B01D09847FA
:102EA00010BD01F0EDF9FBE70000FF1FA222054B6A
:102EB00092009B5810B5002B01D0984710BD01F02F
:102EC000DFF9FBE70000FF1FA322054B92009B5890
:102ED00010B5002B01D0984710BD01F0D1F9FBE7E8
:102EE0000000FF1FA422054B92009B5810B5002B39
:102EF00001D0984710BD01F0C3F9FBE70000FF1FA8
:102F000070B501F085F8514B1860042001F040F9CC
:102F100001F006F80400C30702D401F081F870BD87
:102F200000224B4B1A604B4B1878013804282CD8E0
:102F300000F048FF03231B1F2700200000F0B0FF14
:102F40000128ECD0444C2378042B71D101F068F9AE
:102F5000002806D001F0D4F9582001F089F90223A5
:102F60002370032001F014F9D9E7200001F0F0F8F4
:102F7000E6E7200000F03CFFE2E7200001F060F807
:102F8000DEE7200001F0C4F9DAE700F091FF050068
:102F9000012808D1314B1B78053B012B03D82000B9
:102FA000FFF768FFCEE72C4B1B78022B01D0052BD7
:102FB00020D1022D28D12A4B9B7BAB431CD1200072
:102FC000FFF766FF254B18780128BBD16405B9D4FB
:102FD000234925224B7B034205D1233A13405A4211
:102FE000534126331A000B7D9342ABD9322000F0B7
:102FF00087FFA7E7022D07D1184B1B78052B11D1AE
:103000002000FFF753FFDDE7012D0BD1012B03D18A
:103010002000FFF759FF95E7062B03D12000FFF7AB
:1030200061FF8FE7200001F02BF9022D8AD1C9E75B
:10303000032B04D10B4B987C01F02AF991E7072B65
:103040008FD1094B987B01F08BF88AE79C09FF1F11
:103050009809FF1F9009FF1F2309FF1F1C09FF1F6D
:10306000A60BFF1FBC0BFF1FD40BFF1FFA210A4B3F
:103070000A4A49001A640A4A5A500A4A04395A50FC
:10308000094A08319A64094A5A50094A5C315A502F
:10309000084ADA667047C0460000FF1F7127FF1F0D
:1030A0006D28FF1F2128FF1F7923FF1FE126FF1F27
:1030B000011EFF1FD51DFF1F10B500F06BFE10BDD8
:1030C0008023F7B59C46264B264F01932649274A75
:1030D000274D284C284B02281AD1604638600868D2
:1030E000264E304080263603304308600199097827
:1030F000002909D11660224A2A60224A2260E02271
:1031000019689143A03A1BE08021C9021160F2E7DF
:1031100066463E600F68194E3E408027FF023E43E0
:103120000E600199097800290DD1176001280ED190
:10313000154A2A60154A2260E02219689143C03A74
:103140000A431A60F7BD802189021160EEE7E02191
:103150000F4A02432A600F4A22601A688A43F0E746
:103160004B0AFF1FE0000340D800034090000340DB
:10317000000003405000034040000340FFFFE3FF16
:103180000280063D804508220180063D80660822B7
:103190000080069880550822F8B51E4B80261A68D4
:1031A000002014003440324232D11A681A4F3243A0
:1031B0001A6001223B68063093433B6001F070F8CF
:1031C0000122164D2B681E432E603B680A261343CE
:1031D0003B608027BF00124B1B683B4211D1013E70
:1031E000F6B2FF2E09D17E220E4B1C682B68E40B31
:1031F0001440934323432B6005E0082001F050F86E
:10320000E9E7002EEFD180222B68600893432B6002
:10321000F8BDC046C4F000405CF0004018F000402B
:1032200068F0004060F0004010B500F081FE012120
:103230005820034A00F0A4FEFFF7AEFF10BDC046C1
:10324000600AFF1F10B578220021034800F0C0FF7C
:1032500000F0E6FD002010BD506AFF1F70B50400AD
:1032600000F086FF00230C200B4A010059438D1803
:10327000515C00290DD0A14208D1012300246B70BC
:1032800000F046FE00F024FE200070BD01330A2B42
:10329000EBD11224F6E7C046506AFF1F70B5040058
:1032A00000F066FF002319001D000D4A1078002869
:1032B00006D0A0420CD1557001310C320A29F5D14B
:1032C000002B0AD100F0ACFD00F002FE002070BD22
:1032D0005078461EB0411B18EEE700F019FEF3E7E8
:1032E000506AFF1FF7B504000C20002384460E4DE2
:1032F000019267465F43E85D7E19A04212D0002824
:103300000BD10A4B9C4662461B7808331370019B15
:1033100070707C557160B360FEBD01330A2BE8D13B
:103320000320F9E70720F7E7506AFF1F4C6AFF1FE9
:103330008020F8B5484BC0051B68C1248360474B0B
:10334000FF251A68012313434361454BA4001A6803
:10335000444B40211A60444B1A68444B1A60444B5A
:103360001A59AA431A51C52292009E58AE433143BE
:10337000802699509F583F49F6010F403E439E508A
:103380009E5880273602360A3043985080201A59BA
:1033900000020A4002431A5104341A59364E3F04BF
:1033A000324080263A431A511A5936061202120A3E
:1033B00032431A5108341A5980260A4002431A51DE
:1033C000C32292009F58B446AF4337439F509F5843
:1033D000294E0F4007439F509F58374080263604A0
:1033E000374380269F509F5836063F023F0A374397
:1033F0009F50C0221F59AF433A431A511A59120223
:10340000120A1643C6221E5192009C58AC436546D0
:103410002C439C509C5800250C4020439850C720BA
:1034200080001A58154C1140C02212020A431A504B
:10343000134B1B78DB08AB4201DC0020F8BD23787E
:10344000002B06D0A368002B00D0984701350C3420
:10345000EEE71220F2E7C0463846FF1F3446FF1F52
:10346000B0F00040486AFF1FB4F00040446AFF1FFC
:1034700000E100E0FF00FFFFFFFF00FF506AFF1FB9
:103480004C6AFF1F030010B51F2809D8072200202F
:103490001340072404490A78A24313430B7010BD5C
:1034A00000230620F5E7C0464C6AFF1F034A044983
:1034B000136800200B4013607047C0461CF00040AA
:1034C000FFFFC1FF054B06491B780A6805485B07EB
:1034D00002401B0B134300200B6070474C6AFF1F18
:1034E0001CF00040FFFFC1FF70B50C25FFF7EAFF9D
:1034F0000A4B1C780A4BE4086543ED18002C01D1F7
:10350000200070BD2B78002B06D06B68002B00D0FC
:103510009847013C0C3DF1E71220F2E74C6AFF1F8F
:10352000446AFF1F1FB5002102220B000191009188
:10353000052000F08DFC02230B490A681A42FCD1D9
:1035400020230393039B5A1E0392002BFAD1074AB0
:103550001368002BFCDA0B246C442000012100F0DE
:10356000EFFD207804B010BD90C8004000C80040B6
:1035700013B504000A4B0193019B002B01D11120CC
:1035800016BDFFF7CFFF23000340044205D00520FE
:1035900000F086FE019B013BEDE71800F0E7C04616
:1035A000FFFFFF0707B500F0E3FD80220821D205E9
:1035B000936A0191002B01D10739916202210C4AD3
:1035C00011600199481E01900029FAD10331116060
:1035D000053101910199481E01900029FAD111602D
:1035E000002B02D18022D205936200F071FC07BD4E
:1035F00000C00040F0B52D4C89B02378002B4FD18E
:10360000FEF780F902232A4F03903A681A42FCD150
:1036100020230693069B5A1E0692002BFAD1254EB4
:103620003368002BFCDA0120FFF7A2FF011E02D055
:10363000112009B0F0BD030003220190009005ADF8
:103640009F2000F005FC0321280000F079FD0223F3
:103650003A681A42FCD120230793079B5A1E07920F
:10366000002BFAD13368002BFCDA0120FFF780FF32
:103670000028DDD10398FEF759F9AA786B78110478
:103680001B020B4329780B4363601300113B0A496B
:10369000052B07D801239340A3600B6001232370FF
:1036A0000020C6E780231B03F6E7C0462046FF1F25
:1036B00090C8004000C800409808FF1F1E4B30B55E
:1036C0005A6818781D4B85B0D31859424B410121D7
:1036D0000093002300F094FB194B1A4A02259A63C9
:1036E00000221A6510325A658022C4219D65164B4E
:1036F0001648D202DA6789004258154B80241A40D6
:1037000080231B0413434350642341200393E405A7
:1037100000F006FA402000F003FA6562039D6B1E7C
:103720000393002DFAD103236362FFF73BFFA562E9
:10373000FFF760FF05B030BD2C46FF1F95FFFEF779
:1037400000C80040050001FF04E100E000E100E0E6
:10375000FFFF00FFF0B585B00700FEF7D3F80223A6
:1037600005002D4C22681A42FCD120230093009BB7
:103770005A1E0092002BFAD1284E3368002BFCDA37
:103780000120FFF7F5FE002803D01124200005B02A
:10379000F0BD234B2360022322681A42FCD1202370
:1037A0000193019B5A1E0192002BFAD13368002B22
:1037B000FCDA0120FFF7DCFE0028E6D1194B1F6080
:1037C000022322681A42FCD120230293029B5A1E34
:1037D0000292002BFAD13368002BFCDA0120FFF7AC
:1037E000C7FE0028D1D1104B2360022322681A4261
:1037F000FCD120230393039B5A1E0392002BFAD182
:103800003368002BFCDA0120FFF7B2FE041EBCD1A6
:103810002800FEF78BF8B9E790C8004000C80040C8
:1038200001000006A8C800400180000110B500207A
:10383000FFF790FF10BD000010B5064B18705960DF
:10384000FFF73CFF00211320034AFFF74BFD002048
:1038500010BDC0462C46FF1FBD36FF1FF0B504004B
:1038600085B003920291FEF74DF8882263035B0B4B
:1038700052051A438023DB059D6A8023274F00925F
:10388000BA68002601901B039A420CD9F82326003F
:103890001B041E401C4206D08022214B52025E6255
:1038A00019680A431A60002D0BD100F061FC022256
:1038B0001C4B1A608023DB055A62013A9A6200F0C1
:1038C00007FB0023039A934220D1002D0AD100F078
:1038D0004FFC144B03221D608023DB055A629D625E
:1038E00000F0F6FA8023BA681B039A4208D9002E2A
:1038F00006D000220A4B0C495A621A680A401A6024
:103900000198FEF713F8002005B0F0BD009A029967
:10391000D2181278CA540133D4E7C0462046FF1F9C
:1039200000C8004000C00040FFFFFEFFF0B587B0B8
:10393000029103920400FDF7E5FF019000F018FCEE
:10394000802302250122234EDB0535605D629A62E9
:1039500000F0BEFA204F3B682B42FCD12023049399
:10396000049B5A1E0492002BFAD11C4D2B68002B8D
:10397000FCDA0120FFF7FCFD002802D0112007B07F
:10398000F0BD2000039A029900F082FB022304009C
:103990003A681A42FCD120230593059B5A1E0592D2
:1039A000002BFAD12B68002BFCDA0120FFF7E0FD99
:1039B000051EE3D100F0DCFB80230322DB0535602C
:1039C0005A629D6200F084FA0198FDF7AFFFE0B201
:1039D000D5E7C04600C0004090C8004000C8004085
:1039E000F0B5802489B00600FDF78CFFE405A36ADA
:1039F00002250393029000F0BBFB0123304F3D6092
:103A00006562A36200F064FA2E4C23682B42FCD15D
:103A100020230593059B5A1E0592002BFAD12A4DAF
:103A20002B68002BFCDA0120FFF7A2FD002803D051
:103A30001124200009B0F0BD244B2360022322682A
:103A40001A42FCD120230693069B5A1E0692002B95
:103A5000FAD12B68002BFCDA0120FFF789FD021E4A
:103A6000E6D11B4B03211E60030001900090202033
:103A700000F0EEF9022322681A42FCD120230793BA
:103A8000079B5A1E0792002BFAD12B68002BFCDAF9
:103A90000320FFF76DFD041ECAD100F069FB8023EF
:103AA0000322DB053C605A629C6200F011FA039B22
:103AB000002B01D1FFF776FD0298FDF737FFB8E73D
:103AC00000C0004090C8004000C80040010000064F
:103AD00094C8004007B5000201910422000A01A920
:103AE000FFF724FF0EBD000073B5050005240B4A47
:103AF000A3005B429B1819686B46DE1D300000F086
:103B000087F9022804D133782B55013CEFD276BDDA
:103B1000052CFCD00128FAD10230F8E71409001175
:103B20001F2807D8012380228340D20591680B43C8
:103B3000936070473F2808D80123802220388340B3
:103B4000D20551690B435361F3E75F28F1D8012394
:103B5000802240388340D205116A0B431362E8E7A4
:103B60001F2807D8012280218240C9058B68934312
:103B70008B6070473F2808D801228021203882407E
:103B8000C9054B6993434B61F3E75F28F1D80122E4
:103B9000802140388240C9050B6A93430B62E8E7F5
:103BA0001F2810D880230200DB05153A1968012A66
:103BB00006D820229143196019680A431A60704799
:103BC00001228240F6E73F2811D880230200DB055E
:103BD000353AD968032A06D810229143D960D968AA
:103BE0000A43DA60EBE7012220388240F5E75F28DC
:103BF000E5D842238022181A413B8340D205516AFE
:103C000099435162516A0B435362D8E710B50400DF
:103C1000012813D1A022184992050B685B015B09AA
:103C200013430B60154B164A19681140154A0A4395
:103C30001A60402219680A431A6010BD0028FCD19E
:103C400001000A2000F044FA21000B2000F040FAA5
:103C5000C0220A4B920019680A4340211A601A6870
:103C60008A431A60B022044912060B685B015B09A3
:103C700013430B60E1E7C04614F000401CF0004025
:103C80007F00FEFF80FD010072B6074A1368013312
:103C900013600422054B1A600023054A136080223A
:103CA000D2055360FEE7C0467808FF1FC0F0004011
:103CB000C4F00040044B054A1A60054B1A6000220C
:103CC000044B1A607047C046140AFF1F841E000090
:103CD000380AFF1FC4F000400023034A1360034A60
:103CE0001360034A1360704754F0004040F10040F5
:103CF00044F10040002310B5184C8AB000930193A2
:103D00002378012B27D06946012000F009FA00280A
:103D100017D1009B12490293019B06AA0393114BF2
:103D200002A81B680493104B1B68059300F088FAE7
:103D300010220E4906A800F05BFA002804D1FF23E8
:103D4000237000200AB010BD0123094A074902A8C8
:103D5000237000F075FA0120F4E7C0464C67FF1F9E
:103D600010290011082900110C2900112029001127
:103D70005067FF1F13B501246946012000F0D0F9F8
:103D8000034B00940193FFF7B5FF200016BDC0461A
:103D9000BB0B000010B5FFF79FFFFFF7EBFF0028FC
:103DA00002D0024B984710BDFEE7C046E1A20000DA
:103DB00002B4714649084900095649008E4402BCC4
:103DC0007047C04602B4714649084900095C490081
:103DD0008E4402BC7047C04603B471464908400097
:103DE0004900095A49008E4403BC70470000000096
:103DF00001B40248844601BC604700BF053401009D
:103E000001B40248844601BC604700BFC56D010093
:103E100001B40248844601BC604700BF99380011D4
:103E200001B40248844601BC604700BFADAE00004B
:103E300001B40248844601BC604700BF8D110100F7
:103E400001B40248844601BC604700BF71B0000065
:103E500001B40248844601BC604700BF496D0100BF
:103E600001B40248844601BC604700BFE927000056
:103E700001B40248844601BC604700BF8B52010078
:103E800001B40248844601BC604700BF156B0100C5
:103E900001B40248844601BC604700BFE94C010000
:103EA00001B40248844601BC604700BF01340100F0
:103EB00001B40248844601BC604700BFDD0C01002C
:103EC00001B40248844601BC604700BF19FA0000F3
:103ED00001B40248844601BC604700BF9DA90000B0
:103EE00001B40248844601BC604700BF75F8000079
:103EF00001B40248844601BC604700BF8914010038
:103F000001B40248844601BC604700BF613701002C
:103F100001B40248844601BC604700BF21A90000EB
:103F200001B40248844601BC604700BFBD0B0100DC
:103F300001B40248844601BC604700BFED6801003F
:103F400001B40248844601BC604700BF116E000006
:103F500001B40248844601BC604700BF85C100002F
:103F600001B40248844601BC604700BFE90B010070
:103F700001B40248844601BC604700BFED6B0100FC
:103F800001B40248844601BC604700BF01670100DC
:103F900001B40248844601BC604700BF9D6A00002E
:103FA00001B40248844601BC604700BFB35201001F
:103FB00001B40248844601BC604700BF51B800000C
:103FC00001B40248844601BC604700BF21440000A0
:103FD00001B40248844601BC604700BF851201005D
:103FE00001B40248844601BC604700BF691101006A
:103FF00001B40248844601BC604700BF8944000008
:1040000001B40248844601BC604700BF2D6C01002A
:1040100001B40248844601BC604700BFC95C01008E
:1040200001B40248844601BC604700BFDD0A0100BC
:1040300001B40248844601BC604700BFC1150100BD
:1040400001B40248844601BC604700BFF535010059
:1040500001B40248844601BC604700BF7997000064
:1040600001B40248844601BC604700BF0D52010004
:1040700001B40248844601BC604700BFF9A60000B5
:1040800001B40248844601BC604700BF6D0B0100CB
:1040900001B40248844601BC604700BF957301002B
:1040A00001B40248844601BC604700BFCD0C01004A
:1040B00001B40248844601BC604700BFF90D01000D
:1040C00001B40248844601BC604700BF090E0000ED
:1040D00001B40248844601BC604700BF29A4001116
:1040E00001B40248844601BC604700BFD9B000005B
:1040F00001B40248844601BC604700BFF1B700111B
:1041000001B40248844601BC604700BFD5440100A9
:1041100001B40248844601BC604700BFC16601008B
:1041200001B40248844601BC604700BFE1AC000016
:1041300001B40248844601BC604700BFC9A9000021
:1041400001B40248844601BC604700BF3D710100D4
:1041500001B40248844601BC604700BF0934010035
:1041600001B40248844601BC604700BFC1F70000AB
:1041700001B40248844601BC604700BF75A9000035
:1041800001B40248844601BC604700BFE9D4000086
:1041900001B40248844601BC604700BF1907010012
:1041A00001B40248844601BC604700BF090E00000C
:1041B00001B40248844601BC604700BFA1AF0000C3
:1041C00001B40248844601BC604700BF855201002B
:1041D00001B40248844601BC604700BFB70E00002E
:1041E00001B40248844601BC604700BF53B90000D7
:1041F00001B40248844601BC604700BFCD4C0100B9
:1042000001B40248844601BC604700BF8937010001
:1042100001B40248844601BC604700BF8D820000A3
:1042200001B40248844601BC604700BF01D70000CA
:1042300001B40248844601BC604700BFE9F60000B3
:1042400001B40248844601BC604700BFDD3F000066
:1042500001B40248844601BC604700BFA9D80000F1
:1042600001B40248844601BC604700BF5976010092
:1042700001B40248844601BC604700BF79120100C6
:1042800001B40248844601BC604700BFE917010041
:1042900001B40248844601BC604700BF4DF90000EC
:1042A00001B40248844601BC604700BF0189000098
:1042B00001B40248844601BC604700BFEDA5000080
:1042C00001B40248844601BC604700BFF9ED00001C
:1042D00001B40248844601BC604700BFBD5C0100D8
:1042E00001B40248844601BC604700BFC1A500007C
:1042F00001B40248844601BC604700BFE5120100DA
:1043000001B40248844601BC604700BF6DF600005E
:1043100001B40248844601BC604700BFF935010082
:1043200001B40248844601BC604700BF016C010033
:104330000200000056C1001101000000ECBE001197
:104340000200000052C10011010000007043FF1F75
:1043500002000000F4BE0011010000009064FF1F85
:104360000200000050C10011030000000464FF1FA0
:10437000120000000200000056C100110100000000
:1043800030BF00110200000052C100110100000006
:104390002DBF0011020000003ABF00110300000011
:1043A0003F64FF1F0200000050C100110300000025
:1043B0005464FF1F0200000052C100110100000000
:1043C0002CBF00110200000038BF001103000000E4
:1043D0001564FF1F0200000050C10011030000001F
:1043E0003664FF1F0200000056C1001101000000EA
:1043F00070BF00110200000052C100110100000056
:10440000B944FF1F0200000082BF0011010000003C
:104410006BBF00110200000052C10011010000003A
:10442000B844FF1F0200000080BF0011010000001F
:104430005C64FF1F0200000052C100110100000077
:10444000B744FF1F020000007EBF00110100000002
:104450005BBF00110200000052C10011010000000A
:10446000B644FF1F020000007CBF001101000000E5
:1044700056BF00110200000052C1001101000000EF
:10448000B544FF1F020000007ABF001101000000C8
:1044900051BF00110200000052C1001101000000D4
:1044A000B444FF1F0200000078BF001101000000AB
:1044B0004CBF0011020202020202000000000000D4
:1044C00014130000614D0011274D0011C4BF0011ED
:1044D00090011D0018001800FFFF070102030405EA
:1044E00006020106000000000000000000000000BD
:1044F00000000000000000000000000000000000BC
:10450000030000000200000056C10011010000007D
:1045100044C000110200000052C10011010000005F
:104520007445FF1F020000004EC000110100000092
:104530008A64FF1F0200000050C100110300000048
:10454000F466FF1F0200000052C1001101000000CC
:104550007445FF1F020000004CC000110100000064
:104560008C64FF1F0200000050C100110300000016
:10457000EC66FF1F12006C6C0000000000000000E1
:104580000000000008070000000100000000011109
:10459000FFFF0000504859360000000000000000F6
:1045A00001000000D5BF00110B000500F70000005E
:1045B000B4000028002800283075A000A000A0004A
:1045C000A00000080008E001F0001000100010003A
:1045D000100010001000500050005000100010009B
:1045E000D0070000000000000F000100050030753A
:1045F00007001000010081FF00000000FF00000024
:104600001176001119740011A9710011FFFF01004A
:10461000FF0000002DA00011A99D0011C19C0011F8
:10462000000000000000000000000800040000007E
:104630003B0001085902E00188212800FF0000002A
:104640000200000056C10011010000001CC2001150
:104650000200000052C1001101000000BD46FF1F12
:10466000020000004EC1001101000000086BFF1F96
:104670000200000052C1001101000000BC46FF1FF3
:10468000020000004CC1001101000000BA46FF1FEB
:104690000200000052C1001101000000B846FF1FD7
:1046A000020000004AC1001101000000B046FF1FD7
:1046B000180018001D009001020000030202000013
:1046C0000200000056C100110100000030C20011BC
:1046D0000200000052C10011010000000047FF1F4E
:1046E0000200000048C100110000000000000000AE
:1046F0000200000050C1001103000000286BFF1FE2
:0247000020FF98
:040000051FFF184180
:00000001FF
